S0160000755461736B657256312E345F424D2E7372656358
S10B6080F0170020F5D6000022
S113609008B561202A2102F0CEFC08BD08B56120B4
S11360A0292102F0C8FC08BD08B5134B188020282C
S11360B00ED004D800281BD008281CD118E0802852
S11360C016D080235B00984208D0402813D10FE0FB
S11360D061200A49062203F021F80CE0062261201F
S11360E0074903F01BF8074B1A78074B1A7002E0B4
S11360F0612003F04DF808BD0CF9FF1F983A000029
S1136100B80B0000E4F8FF1FCCF8FF1F37B5214D92
S113611021482968402204F042FA00280FDA1C20A2
S11361202968402204F03BFA0024A04209DA2868D6
S11361301A494022802407F0EFF8E40101E08024AA
S11361402402286803781B2B04D01449402207F04A
S1136150E3F80024124B29681868402207F0DCF8A1
S113616080231B029C420CD169461C20073101226A
S113617004F015FA00280BDA022004F028FA0024AF
S113618006E08023DB019C4202D1002000F0BCFB2E
S1136190201C3EBDE8F8FF1F1C80000028DA000028
S11361A0E0F8FF1F08B5084B084A19781170002859
S11361B004D0022805D102F0F5F904E0044A12786B
S11361C000E0FF221A7008BDCCF8FF1FC0F8FF1FC3
S11361D0E4F8FF1F024B1A78024B1A707047C0464E
S11361E0C0F8FF1FCCF8FF1F30B51C4B85B01B68EF
S11361F0011C0024684604721A7BC2722022828029
S113620080225200C280612202731A1C3632127834
S113621082731A1C37321278C2735B686A46009321
S113622001234373201C02F05FFB0D4D2870A04234
S113623010D0221C052102F005FA009A520609D555
S11362400849221C287802F0FDF928788121221CB3
S113625002F0F8F9287805B030BDC046E8F8FF1F11
S1136260E4F8FF1F04040000F0B5784D91B02C68E9
S1136270867B002C65D1201C04F022FE402002F015
S113628073FD734B1860402002F06EFD714B186073
S1136290201CFFF73BFF80231B02984201D00123FF
S11362A02B6000F01DFD6D20042102F001FF03208E
S11362B0FFF79AFF002800D1C5E0674B67481A78BA
S11362C0674B02271A7002F0D9FB7520042102F0F3
S11362D0EFFE644B6946009301234B7109228B73D3
S11362E00293684612230A718B8106F097F95E4B7C
S11362F0684600936B469F7340230293FA2406F08A
S11363008DF9694603230B710C224B71BC40C823E1
S113631068468A72CB800C8106F080F96A46577110
S11363208023927A5B42134369468B724F480B89F0
S1136330211C584307F000FB6A46D080684606F0EB
S11363406DF94B4F301C6946052202F091F9002883
S113635040D06B46DC781A79002C02D0012C0FD087
S113636032E0D2B2062A04D0832AEBD106F0CAFF67
S1136370E8E7394916220878391C02F04DFBE1E7B9
S1136380B72A06D0DD2A09D12A68082ADAD12C6076
S1136390D8E7201C06F04EFF364812E0283AD2B265
S11363A0042ACFD8344802F069FB69460B79292BBB
S11363B006D02A2BC6D1201C06F03CFF2F4800E053
S11363C02F4802F05BFBBDE792B2301C694602F035
S11363D04FF9B7E72A6837231A4234D01E4D28787C
S11363E002F056F900282ED0264F2878694640221C
S11363F002F03EF9041E26D0234A80261388F601B3
S11364001E406846211C002E02D002F0BFF8ECE7C3
S113641000F03EF93A886846211C002A0FD101F0A9
S113642011FC0028E1D08020400000F0FFFA02288F
S1136430DBD128781549172202F0EEFAD5E7321C91
S113644001F000FCD1E711B0F0BDC046ECF8FF1F2D
S1136450E8F8FF1FE0F8FF1FE4F8FF1F68DA000008
S1136460CCF8FF1F9D60000091600000C202000094
S113647010DA000085DA000097DA0000B5DA0000CF
S1136480A0DA00000CF9FF1F00F9FF1FCBDA0000AF
S1136490704700B50A78031C002A06D01B78013126
S11364A001309A42F6D000200CE000214156202908
S11364B007DC00229A56202A01D10133F9E7181C7F
S11364C000E0101C00BD70B50368021C0021595681
S11364D0202904D11168013301311160F6E71D1D33
S11364E000200F26AB4215D019784CB22F2C11DDA9
S11364F0CCB2211C30390001C9B280B20133092960
S113650002D9211C3739C9B231400843116801311D
S11365101160E7E770BD00B5036800229A56202A8F
S113652005D020211A788A4301D00133FAE70022EA
S11365309A56202A01D10133F9E703600020185646
S11365404342584100BD838802685BBA838013BA12
S11365500360704708B5054802F090FA044802F059
S11365608DFA044802F08AFA08BDC0462BE0000008
S113657062EC00003EE00000F0B52C4A2C4E13788B
S11365800C2253439C59F3181A798BB0071C0192BF
S113659003A820211B225D7906F05CFF002F04D0A4
S11365A0BD4210DD0C34013DFAE7224802F066FAE0
S11365B01E4A13780C225343F618B06802F05EFAB0
S11365C01D4802F05BFA1D4E1D4F002D29D0307876
S11365D00021422202F020FA002808D1307840211C
S11365E0184A02F02FF8184B01201D601CE02068A7
S11365F002F044FA019B021C30789A4202DB03A9A0
S1136600012203E0019B03A99A1A92B202F004FA50
S1136610606802F033FA381C02F030FA0C34013DA1
S1136620D3E7094B281C1D600BB0F0BD1DF9FF1FFB
S113663040DE00003DE0000041E00000CCF8FF1F18
S11366403EE000006D10000004F9FF1F30B50F4D4F
S1136650847B89B0201C6946052202F009F80028D1
S113666012D06946CB780A79012B07D1DD2AF1D102
S113667028680028EED0FFF77FFFEBE792B2201CDA
S1136680694601F0F5FFE5E709B030BD04F9FF1FE5
S113669008B50A1C0349031C0878191C02F0BCF94C
S11366A008BDC046E4F8FF1F154B164A1B68126864
S11366B05868516810B50124884208D1D88ED18E0B
S11366C0884204D1117B1C7B641A611E8C4152895F
S11366D05B8953402822134201D00222144304222E
S11366E0134200D01443DA0601D508231C430120C9
S11366F0FFF70CFDE30702D50420FFF775FD10BD7D
S1136700E8F8FF1FE0F8FF1F08B5034B03491868BA
S1136710402206F001FE08BDE8F8FF1F28DA000059
S1136720F0B5694C89B0039020680591032800D91D
S1136730A5E007F09FF8022C289C644D2B68002BE1
S113674005D180208000042102F032FB2860604AD9
S1136750002313605F4A13605F4B2A681A600123A9
S1136760236014E05D4A08335D48136003F05EFF64
S11367705C4B186002235C48236002F07FF9301CF4
S1136780FFF7E1FE0395039C514D534E6AE0524FCF
S1136790039D3A6801924E4A0199136894465A42FD
S11367A0524EB34230D8059E002E04D14A4A11609D
S11367B0474A136085E0039801318618F65C013579
S11367C00496019E0498B618F054059801330138D4
S11367D080B20590082BE3D1396061460B603B4BD6
S11367E01E68301CFFF7AFFEB288414B9A4201D0BD
S11367F0404804E03368404A9342B3D93F4802F02A
S11368003DF9032323605CE0334A1160304A13608E
S1136810B8E7059A0398811889B2A2B291422ED0A2
S113682032680133511C04933160049821782B6041
S1136830802311709B00984213D1314802F01EF955
S1136840284B224F18683968049A03F04BFF214BF8
S11368508020196880000A183F681A6000232B60A2
S1136860376001342B68214A9342D2D907E0039E52
S1136870002E26D1059E002E23D1266021E0154B43
S11368801349164A1B68096812685918914218D3AB
S11368906C461F3405212170124D9A4205D90B49CB
S11368A0D21A0968286803F01DFF211C286803F028
S11368B0BFFF144802F0E2F861206421832202F051
S11368C02DFC09B0F0BDC04608F9FF1F10F9FF1FE9
S11368D014F9FF1F18F9FF1FF8F8FF1FFCF8FF1F3A
S11368E08DE0000020F9FF1F8FE00000FF01000091
S11368F03412000059E00000FF7F000073E0000044
S11369009DE000009FE0000038B50A4C051C21689A
S11369100948402203F022FE012D08D0022003F092
S113692056FE064B21681868402206F0F5FC00204C
S113693038BDC046E8F8FF1F1C800000E0F8FF1FC8
S113694008B5044B021C1B680A21D86B02F09EF8A0
S113695008BDC046E8F8FF1F7FB5054802F08EF871
S113696001A8FFF7EDFF01A802F088F807B000BD09
S1136970BAE000007FB5031C02380B2845D806F0A6
S113698079FF0644114444443A351825182DFFF77D
S1136990E3FFFFF7DFFD1E4802F070F81D4B186897
S11369A0213020E01B4B14221868213006F0B4FC7F
S11369B02BE00C3B581E83410420C01A01A904F0AB
S11369C0D9F801A802F05AF813480CE0102004F09A
S11369D0D1F8124802F052F80C2013E010200021E4
S11369E004F0C8F80E4802F049F80EE0082004F05C
S11369F0C1F80C4803E0202004F0BCF80A4802F077
S1136A003DF80A200021FFF7B5FF07B000BDC046DE
S1136A10CCE00000E8F8FF1FF7E20000E4E000002B
S1136A20F4E0000004E1000013E10000802310B54D
S1136A305B0098420FD08022234B1201904216D162
S1136A401B880224002B3CD1204B1B88002B38D1FF
S1136A501F4B18800EE01E4B02241B88002B30D1E4
S1136A60194B1B88002B2CD1FFF71EFB02E0802260
S1136A7092001A80154B1A8880235B009A4203D136
S1136A802020FFF711FB0AE0114B80221988120124
S1136A90914204D1802252011A8001F083FDFFF754
S1136AA05BFFFFF757FD0B4801F0E8FF0A4B00249A
S1136AB01868213001F0E2FF084B201C1C70FFF71E
S1136AC05BFD201C10BDC046F0F8FF1F0CF9FF1F32
S1136AD000F9FF1FCCE00000E8F8FF1F1DF9FF1FBD
S1136AE0313800B5002303282ED8184B1849194A09
S1136AF006F0C0FE020C1620186809681B681268AC
S1136B009A43031C0B4013439B061CE01868096856
S1136B101B6812689A43031C0B401343DB0612E004
S1136B20186809681B6812689A43031C0B401343D6
S1136B305B0608E0186809681B6812689A43031C1E
S1136B400B4013431B06DB0F181C00BD94F00F40D1
S1136B5080F00F4090F00F40F7B5134F01253B68CC
S1136B6031201A1C38321278002400925B8F019372
S1136B70461C40B2F6B2FFF7B3FF002800D02C4306
S1136B806D00EDB2392E01D0F0B2F1E7FFF78CFDC4
S1136B903B6800991A1C383211705470019A002015
S1136BA05A87FFF7B1FEF7BDE8F8FF1F031C313B1E
S1136BB000B50020032B10D8084A181C12680123C2
S1136BC006F058FE02040608520904E0120902E025
S1136BD0920900E0D209181C904300BD94F00F40C4
S1136BE038B5031C303B0020032B4ED8181C06F08C
S1136BF041FE02080406202404E0402402E080242C
S1136C0000E010245DB264290BD003DC002061296C
S1136C103BD003E0692904D06F291CD001204042F5
S1136C2033E01A4B8022196812010A431A60184B88
S1136C3002201A68211CA2431A600422FF3205F0C4
S1136C40CDFC144B1A680123AB4038321D1C137859
S1136C50AB43137018E00D4B8022196812010A43EC
S1136C601A608222211C5200022005F0B7FC084B56
S1136C701A6814431C60074B1A68012338321178D0
S1136C80AB401D1C0D431570002038BD38800440F6
S1136C9094F00F40E8F8FF1F00B5002905D00E4B13
S1136CA08022196812010A431A60012303405B0120
S1136CB0820701D510221343420701D54022134312
S1136CC0020701D580221343044AF020116881434E
S1136CD00B43136000BDC0463880044080F00F4071
S1136CE0F7B5AF4D01212B6801241A1C3832393312
S1136CF01778187838401870FFF7CEFF30206921D4
S1136D00274200D06F21461C49B240B26400F6B25B
S1136D10FFF766FFE4B2382E01D0301CEFE76120A4
S1136D20461C40B26238F6B29E4B0E2809D806F0D3
S1136D30A1FD1018202F353D454D555D656D7C8DA9
S1136D4095001968802252010A4380241A60640065
S1136D5016E01968802252010A4380241A60A400B4
S1136D600EE01968802252010A4380241A60E4006C
S1136D7006E01968802252010A4380241A60240123
S1136D8082220320211C520005F028FC864B73E06C
S1136D901A688024640122431A60F1E7196880228A
S1136DA052010A4380241A60A401E9E71968802289
S1136DB052010A4380241A60E401E1E71968802241
S1136DC052010A4380241A602402D9E719688022F8
S1136DD012010A4380241A60640146E01968802283
S1136DE012010A4380241A60A4013EE0196880223B
S1136DF012010A4380241A60E40136E019688022F3
S1136E0012010A4380241A6024022EE019688022A9
S1136E1052010A431A60822208215200032005F01D
S1136E20DDFB614B08211A680DE0196880225201CC
S1136E300A431A60822210215200032005F0CEFB7F
S1136E40594B10211A680A431A6018E01968802205
S1136E5012010A4380241A60E40206E019688022C1
S1136E6012010A4380241A60240382220220211C76
S1136E70520005F0B3FB4D4B1A6814431C60712E8D
S1136E8001D0F0B24CE72B6880215B8F8020484A08
S1136E90484C01931025012309020001019E1E4262
S1136EA066D0802B50D016D8082B44D009D8022B9A
S1136EB039D0042B3CD0012B00D0C5E080267600CD
S1136EC033E0202B3AD0402B3BD0102B00D0BBE03A
S1136ED08026760129E083423ED0802683420ED864
S1136EE0B600B34232D08026F600B34231D08026B9
S1136EF07600B34200D0A7E08026760133E0B601E5
S1136F00B3422CD006D880267601B34200D09BE051
S1136F1008260AE08026F601B34222D080263603F2
S1136F208B4220D090E08026B600B446224E1CE06E
S1136F308026F600F9E7204E306085E08026B60111
S1136F40F3E78026F601F0E71B4E06E08026B60143
S1136F5009E08026F60106E0184E316074E0102640
S1136F60E3E78026F602B446144E674637606BE0CA
S1136F70802B59D024D8082B4ED008D8022B45D0CA
S1136F80042B46D0012B5FD18026760057E0202BBE
S1136F9044D0402B45D0102B56D1802676014EE0AC
S1136FA0E8F8FF1F38800440D4F00F4094F00F40FD
S1136FB0C8F00F4088F00F40C4F00F4084F00F4039
S1136FC0834239D0802683420DD8B600B3422DD0F7
S1136FD08026F600B3422CD080267600B34233D10B
S1136FE0802676012FE0B601B34227D005D880264B
S1136FF07601B34228D1082621E08026F601B34267
S11370001FD0802636038B421DD01DE08026B6009B
S113701015E08026F60012E0106015E08026B60127
S11370200DE08026F6010AE011600DE08026B6012D
S113703009E08026F60106E0216005E010261660CE
S113704002E08026F60226605B00013D9BB2002D23
S113705000D023E7F7BDC04670B52E4B041C1A7848
S113706052B2002A30DB1A7802210A422ED1187853
S1137070042210422CD1187885062BD41E780120C6
S113708040251B78064203D02B4225D0224934E008
S11370902B4223D1214B1D78054221D11878084277
S11370A020D1197811421FD11A7811071ED41A1C45
S11370B01B78DD061CD4137899061BD413785BB2B5
S11370C0002B19DA164918E0164916E0164914E09F
S11370D0164912E0164910E016490EE016490CE074
S11370E016490AE0164908E0164906E0164904E084
S11370F0164902E0164900E01649002C04D1081C88
S113710001F0BCFC201C04E0201C01F0EFFD001B7E
S1137110C0B270BD00F0074024DB000001F007405E
S113712060DC00004FDF0000C4DE00003DDC000036
S11371305DEC0000FCDA000034DC0000E3DB00005E
S11371402DDC000024DC0000DCDD000024E0000075
S1137150D0DB00001CDB0000F8B506F05FF8164E2B
S1137160164F051C0024601E072805D806F082FB74
S113717006080A0C0E101214301C0EE010480CE025
S113718010480AE0104808E0104806E0104804E0FF
S1137190104802E0104800E0381C01F06FFCA542E2
S11371A002D10E4801F06AFC0D48013401F066FC7E
S11371B0092CD8D1F8BDC04622E100006AE10000E4
S11371C02AE1000033E100003CE1000045E1000059
S11371D04EE1000056E1000060E1000074E10000AF
S11371E0F7E20000F0B50C1C95B0151C082801D975
S11371F000F0DFFC06F048FB09003900CB02E7028F
S1137200DD044503C204C704AB02081E05D00429EB
S113721008D10122C04B00201A70FFF7ADF9041CFD
S113722000F0D5FC02220529F4D003220629F1D06E
S113723004220729EED005220929EBD006220A29C7
S1137240E8D007220E29E5D008220F29E2D009222E
S11372501029DFD00A221129DCD0122901D000F034
S1137260A8FCAD4B00201870D7E70892202901D95B
S113727000F09FFC081C06F007FB21003800CB003F
S11372809C04B8007A009C049C049C049C0459004F
S11372906300B5009C049C04E200D401D4019C0466
S11372A09C049C049C049C049C049C049C04250055
S11372B0E200D401D4014A022D00310006F022F884
S11372C000F077FC954801F0D9FB0020FFF7C4FEDD
S11372D000F06FFCFFF740FF00F06BFC002010563D
S11372E0303805F0A7FF00F064FC8D4801F0C6FBC0
S11372F08C4801F0C3FB8C4801F0C0FB01F098FD01
S1137300822101F08FFC894801F0B8FB01F084FD73
S1137310822101F087FC864801F0B0FB01F06EFD8C
S1137320822101F07FFC834800F03CFC0AA803F0B2
S1137330F7FD00240470804801F0A0FB0AA801E2D4
S11373401378313BDBB2032B02D97C4800F02AFCD2
S11373507B4801F093FB089900200856FFF726FCB0
S1137360041E01D17748EDE1774800F01BFC10784A
S1137370031C313BDBB2032B02D9744800F012FC2E
S113738040B2FFF713FC041E02D0714800F00AFC5F
S1137390051C01263120471C40B2FFB2FFF7A0FBB9
S11373A0002801D03543EDB27600F6B2352F01D076
S11373B0F8B2F0E7089801F03EFCC6B20898013E26
S11373C00123B34001301E1C089001F034FC012855
S11373D001D1354300E0B543E8B20021FFF75CFC7E
S11373E000F0F5FBFFF7B8FBE3E31378313BDBB2C6
S11373F0032BC2D8574801F041FB089A00201056CD
S1137400FFF76EFB041E01D05348CBE3534899E1C8
S1137410101C099201F00FFC041C09A8FFF77BF86B
S1137420002801D04E48BDE3099B2F34002160B2EF
S11374305956FFF7D5FB002800D1BAE3F2E7002341
S1137440D356002B02D11027039727E0101C01F01C
S1137450F2FB444B186008A8FFF75DF8089B1A7804
S1137460002AF0D020218A4352B204214C2A02D0AF
S1137470572A04D102213C4A0133116005E0422A13
S113748004D1394A012111605B180893089800233C
S1137490C356002BD7D001F0EAFB0390334801F028
S11374A0EDFA0AAB20222F4D1A705A70039F002F59
S11374B000DC7EE3286884216F4601F0B3FB2A37A1
S11374C02B4801F0DBFA0197274E10270497039FFE
S11374D03268013F0397022A14D0042A53D0012AA8
S11374E000D066E31B2C07D16F461E372868391C71
S11374F005F066FF3B7801E0286803780993099951
S1137500C8B23CE01B2C35D16F461E372868391CA5
S113751005F056FF3B882FE01DF9FF1F7EE10000B8
S113752092E1000044E00000A9E10000B6E100009F
S1137530BDE100003EE00000CFE10000F4E1000006
S113754006E2000019E2000022E200002AE2000044
S113755039E2000049E2000056E200005AE200006D
S11375605EE20000F4F8FF1FC8F8FF1F66E20000A7
S113757077E200002A6813880993099B98B233784C
S1137580102119430DE01B2C04D1286809A905F02A
S113759017FF02E02B681B680993337810210998C0
S11375A0194301F03FFB2F6833680998DA19049FE7
S11375B02A60FF1A04970290022B06D0191F484232
S11375C04141182249420A4000E008220199CF189B
S11375D00597059881420FD00298D040009020383A
S11375E0C0B2844667462E205A2F01D8009FF8B2B5
S11375F00870083A0131ECE7019FFF180197039FD7
S1137600002F03D0049F002F00D060E7019F0D23BB
S11376103B700A237B700023BB700AA801F02EFA8A
S113762044E70023D356002B00D1C2E2101C01F022
S113763002FB051C112C01D01D2C01D1B74800E020
S1137640B74801F01BFA08A8FEF765FF089B1A78F3
S1137650002A00D1ADE220218A4352B204214C2AEF
S113766002D0572A04D10221AE4A0133116005E049
S1137670422A04D1AB4A012111605B18089308A87F
S1137680FEF749FF089801F0D6FA0A9008A8FEF719
S113769042FF112C02D001231D2C08D1089800228E
S11376A082560123002A02D001F0E1FA031C1C3C9B
S11376B0E4B2002601229B4FA24276411C1C002CFE
S11376C000DC76E23A68022A0BD0042A14D0012A9C
S11376D019D10A9B002E02D009A90B7006E02B7069
S11376E011E00A9B002E05D009A90B80281C05F087
S11376F00FFF08E02B8006E0002E02D0281C0AA908
S1137700F5E70A9828603968013C6D18D7E700232B
S1137710D356002B00D14CE2101C01F08CFA041C4F
S113772008A8FEF7F8FE08980022825600218A4233
S113773002D001F080FA011C201C04F035FE041E66
S113774003D1794801F09AF941E278482AE2002904
S113775002D001290AD02CE2754801F08FF9754B4B
S113776080221988D2010A431A8030E2714C8023A6
S113777022885B019A4201D06F4813E26F4801F0FE
S11377807DF9228880239B011343238011E2002981
S113779009D0032900D00CE2694B101C1C6801F0CD
S11377A066FA208105E2674D2B88042B05D16648D3
S11377B001F064F910232B8009E25E4B081C198048
S11377C0FEF772FC03E20A92072900D9F1E1081CD2
S11377D006F050F804244148134D52380AA8FEF725
S11377E072FE041C0AA8FEF76EFE09A908700122A5
S11377F0201C02F0B3FE5548D4E10AA8FEF763FE4C
S1137800041C0AA8FEF75FFE09A90870504801226B
S11378100443A0B202F0A2FE4E48C3E10AA809AC98
S1137820FEF751FE211C012202F0B9FE002807DBFD
S1137830494801F023F92078092101F0F3F9B8E16E
S11378404648AFE13E4B40221868454B196805F0A5
S113785063FD4448A6E1FEF757FF0020FFF754F804
S113786041489FE1012002F0B2FE40489AE1022023
S113787002F0ADFE3E4895E10020FFF745F83D4893
S113788090E11D2900D994E1081C05F0FDFF1E00BC
S1137890990031007B00B60092019201920192019D
S11378A0920192019201920192019201920192013C
S11378B0D400920192019201470147019201920181
S11378C09201920192015B0171011D4B2A4F1E68C6
S11378D00024E000001B3818291C01F0EDF90028F1
S11378E001D1347362E101340C2CF2D1234859E103
S11378F00023D356372B05D1114B01221B685F6837
S11379003A4307E0382B07D10D4B01221B68586816
S11379109043021C5A6049E1194843E17CE20000AB
S113792083E20000C4F8FF1F8BE2000094E2000031
S1137930A4E2000000F9FF1FDCE20000FAE200000C
S1137940E8F8FF1FF0F8FF1F11E300001DE300003B
S11379500080FFFF2FE3000047E300005CE300002A
S1137960E0F8FF1F7EE300009FE30000BFE3000098
S1137970DAE30000F7E30000D1DE000009E50000CF
S11379800FE40000934B944F1E680024A0000019DC
S11379903818291C01F090F900280CD171680623CD
S11379A099430B1C002C04D0012C00D0FDE00222D2
S11379B03AE0042238E00134032CE7D18748F1E0AF
S11379C0844B874F1E680024A0003818291C01F03E
S11379D073F900280CD1726818239A43131C012CE4
S11379E004D0022C00D0E0E010221DE008221BE0AD
S11379F00134032CE8D17B48D4E0764B7A4F1E68DF
S1137A000024E0003818291C01F056F900280DD193
S1137A10776860239F433B1C012C04D0022C00D0C8
S1137A20C3E0202200E040221343BEE00134032CD3
S1137A30E7D16E48B6E06E4801F020F86D4801F0D9
S1137A401DF8644C2068037B0B2B04D8D800C31AA0
S1137A506948C01800E0694801F010F8684D281C16
S1137A6001F00CF823682E1C5B68D90701D5654822
S1137A7000E0654801F002F8644800F0FFFF236865
S1137A805A680123970704D404231A4053425341EC
S1137A905B009800C3185048C01800F0EFFF5C4822
S1137AA000F0ECFF236802205B68D90601D41807B4
S1137AB0C00F4B4B8000181800F0E0FF554800F051
S1137AC0DDFF236801255B685A0602D49D06ED0F8D
S1137AD06D00514800F0D2FF4348EB00C01800F09D
S1137AE0CDFF301C00F0CAFF002D62D04B4800F0DF
S1137AF0C5FF236800213633187801F041F8484D5A
S1137B00281C00F0BBFF474800F0B8FF23680021A1
S1137B103733187801F034F8281C43E0101C01F0C6
S1137B20A6F8C0B2632803D8002802D1012000E0DF
S1137B306320284B1B68152C01D1363300E0373302
S1137B40187033E0384800F099FF384800F096FF89
S1137B50012005F0C5FC182101F012F8344800F0AA
S1137B608DFF002005F0BCFC182101F009F820E08D
S1137B700120404205F0B4FC2E4813E0081C111CFF
S1137B80FEF7F8FE15E0062913D12B48111C01F06D
S1137B9093F8041E0FD02948291C01F08DF8041E07
S1137BA00FD0274800F06AFF03E073600420FEF75B
S1137BB01BFB00240BE0074B40211B685A890A4336
S1137BC004E0044B40211B685A898A435A81201CD3
S1137BD015B0F0BDE8F8FF1F40DF000022E500000B
S1137BE0C4DB000035E500000CE000004BE50000BC
S1137BF027E4000040E40000D1DE000048E4000077
S1137C00F7E2000051E4000053E4000055E40000F2
S1137C102BE500005DE400006CE400007AE4000061
S1137C2086E400008AE4000095E40000AAE4000071
S1137C30BBE40000CCE40000E7E40000EEE4000054
S1137C40F6E40000F0B587B005910021071C04920A
S1137C5003910599002900D104E13B78082B0DD14B
S1137C60824B1A78002A05D08148013A01301A70F3
S1137C7000F004FF7F4A00231370EEE01B2B01D1B8
S1137C807C4905E05B2B06D17A490A781B2A02D18C
S1137C900B700137E1E077490A785B2A4BD1181C55
S1137CA04138032847D805F0E5FD101009026F4B51
S1137CB01A78002A00D1D0E0013ACDE06B4B1A7853
S1137CC0272A00D9C9E00132C6E06B4C282022687B
S1137CD06A4E5043301801F015F83B78051C412BCF
S1137CE008D12368002B01D1032300E0013B23606A
S1137CF0634806E023680133032B00DD0023614859
S1137D00236000F0BBFE002D04D05F4800F0B6FEF7
S1137D10013DF8E75B4800F0B1FE20682825684380
S1137D20301800F0ABFE20684543701900F0EAFFFC
S1137D304E4B187091E00A2B00D18EE0002B00D13D
S1137D408BE04D4928250968484C02916943227803
S1137D504A4E89188B553B780D2B72D10A2304980F
S1137D608B55FEF71FFA444A0C20126823785543BA
S1137D70464A474912780133424375195458DBB2D5
S1137D808A185679EA180021013A117004990029D9
S1137D9006D1404A1288002A41D0510507D53EE059
S1137DA0049A022A03D13C4A1288002A37D0002BB5
S1137DB032D0281C002E19D02168FEF76AFB013E40
S1137DC00390002810D0354800F058FE207A617ADC
S1137DD0039AFFF707FA002802D1314800F04EFE5B
S1137DE0049B002B1BD112E00C34E2E72D49FEF773
S1137DF050FB021E10D004200921FFF7F3F90028DC
S1137E0002D1274800F03AFE0499002907D1214BFA
S1137E101888FEF749F902E0234800F02FFEFEF728
S1137E20D9F9124B00221A70134B19680131032936
S1137E3003DC01221960039205E01A600123039315
S1137E4001E0013222700B4B00221A70074B0137FC
S1137E501A78272A01D927221A70059B013B9BB265
S1137E600593F6E6039807B0F0BDC0461EF9FF1F60
S1137E7020DB00001CF9FF1F24F9FF1F28F9FF1F56
S1137E8064E500003FE000007AE200001DF9FF1FF6
S1137E9040DE00000CF9FF1F00F9FF1FF7E20000AD
S1137EA062E2000068E500005EE2000038B5051CEF
S1137EB02A1C002000F018FD041E10D00521002209
S1137EC000F0C0FB2B685A0609D506490022201C85
S1137ED000F0B8FB201C8121002200F0B3FB201C21
S1137EE038BDC04604040000F0B585B069460A23D5
S1137EF0CB7220238B8080235B00CB8075230B7394
S1137F0050238B731423CB73002300930123041C8D
S1137F104B73164D164F174E17D10B72684603213B
S1137F20FFF7C4FF6A466870D37A03213B70009B55
S1137F306846336002231372FFF7B8FF6946A870DE
S1137F40CB7A009A7B7072600EE0431EFA5C69463D
S1137F50CA729A00B658084A6846D35C00960B72F7
S1137F600421FFF7A3FF285505B0F0BD00FAFF1F59
S1137F70D4F9FF1FD8F9FF1FC9ED0000F7B5041CA1
S1137F800D1C161E04D00020022A77D0021C3DE0EE
S1137F9002788023111C9943042021296ED1E179B0
S1137FA0A779374B0902394352B21980002A11DAF2
S1137FB01E806378212B61D16179237909021943E9
S1137FC0304B7520196049100A31C9B200F033FDF5
S1137FD0321C15E06378202B09D0222B4ED1627914
S1137FE0237912021A43274B1A60032208E0264A17
S1137FF013706279237912021A43224B1A60062203
S1138000101C082D3AD9083DADB208341C4B101C85
S11380101988002932D01C4B1A78202A20D1194BF8
S11380201B68DE0FF6187610184BF000801B18182A
S11380300B1C072900D907239FB22A1CBD4200D973
S11380401A1CC01B92B20730211C019205F064F97E
S1138050019BBB4204D31436F1B2752000F0EBFC53
S1138060094900220A7006490B889D4202D30A80FE
S1138070032003E002495D1B0D800620FEBDC046BF
S1138080CCF9FF1FD0F9FF1FF9F9FF1FE4F9FF1F17
S1138090F0B5CE4B807B1A78A9B00190002A00D0AD
S11380A08EE0CB4B04261D682135281C00F02AFEE7
S11380B0440001D0A61CF6B2C64F3B68002B06D183
S11380C0301C00F051FE03233860067043703B6897
S11380D0002C02D00233002102E09C70DC7007E027
S11380E02A78002A04D01A70597001350233F7E750
S11380F00020FFF7F9FEB84B002503AA01267527D7
S11381000393291C0823052056811674537497740D
S11381109573D580958000F0E7FBAC4C102320705C
S113812008AC63818023B340A774E6734027A67329
S1138130291C8026221C0520A781A780E380268194
S1138140089500F0D1FBA54E03233070A780291CAD
S11381508027221C0520A373E373E78000F0C4FB8F
S113816005277070291C221C381CA773E77300F0C4
S1138170BBFB0223B070291C221C381CA37365812D
S1138180E573A5740895A580E58000F0ADFB944ED9
S113819004233070291C221C381CA37300F0A4FB98
S11381A006237070291C381C221CA37300F09CFB4E
S11381B0B07005E0E378012B0BD0752B00D130E1D2
S11381C008AC0198211C052200F052FA0028F1D1D4
S11381D03CE12279CB2A18D0CC2A07D0CA2A28D14C
S11381E00220002101F0B0FE7E482CE17E4C238861
S11381F0002B08D07D4B00201A787D4B1A70FDF7B8
S113820053FF002323807B481DE1774C2388002BF8
S113821009D0764B00201A78754B1A70FDF744FF8D
S1138220714D00232B800120002101F08DFE724846
S113823009E1132A00D882E0101C14386F4CC100E5
S11382400E1A355DA61973781B029C46B3786746EF
S11382501B043B43F7782B433F06E1261F43B6023A
S11382600C23B74236D8E1260B237602B74231D825
S1138270E1260A233602B7422CD896260923360271
S1138280B74227D896260823F601B74222D8E1261A
S11382900723B601B7421DD8062396269E40B7424F
S11382A018D8052396269E40B74213D80423962651
S11382B09E40B7420ED8032396269E40B74209D863
S11382C0022396269E40B74204D896235B00BB4205
S11382D09B415B420E1AA619B7797679073F7D4216
S11382E07D41AFB2012E02D0022E02D100E004265D
S11382F03743091A64182179012903D0022903D1CB
S1138300102100E008210F4300280BD1304A1F211F
S113831012680420566813738E4337435760FDF781
S113832063FF4DE7153A3649940066581F25AE435E
S11383303743675033498B54FFF7D6FD40E7092A8A
S113834000D83DE7131C0A3B002B04D1204A1268D5
S1138350117B506805E02B490B3A2948895C92004F
S113836010580C2903D8284A89008E5801E0962613
S1138370F6012249DA00D41A6654370A0C19360C6D
S1138380A67000266770E670C60701D5072600E0D0
S11383900826A6710224204207D10424044004D0F4
S11383A0D41A0C190126667102E0D61A8E1974715A
S11383B0070703D5D01A0818012405E0102420402B
S11383C024D0D01A08180224047122E0E3F9FF1F14
S11383D0E8F8FF1FFCF9FF1F7D7F0000C8F9FF1FAD
S11383E0E0F9FF1FA1EC000000F9FF1FE4F8FF1FF4
S11383F0CCF8FF1F85EC000091EC0000E4F9FF1FAE
S1138400D8F9FF1FD4F9FF1FD0ED0000D41A0C19BE
S11384102071554CD31A2078C918072200F0FCFAB1
S1138420CEE6694622790198253100F021F9637975
S1138430FE2B00D0C4E64D4800F020FBA0790121BA
S113844000F09EFB4A4800F019FBB9E6494D287834
S113845000F01EF92E1C00281DD0474FC0223B8877
S1138460D201134224D0580418D5444F002138783F
S1138470402200F0D1FA002808D0211C402228789C
S113848000F0F6F8211C021C387830E038784021DE
S11384903B4A00F0D7F801253A4F2EE0211C2878FA
S11384A0802200F0E5F8011C201CFEF739F9CEE724
S11384B0211C8022287800F0DBF8061C211C321CC9
S11384C0287800F0A9FA2C4F201C3B88311C02228A
S11384D0002B0FD1FFF7B6FB0028B8D08020000195
S11384E0FEF7A4FA0228B2D128782749172200F00F
S11384F093FAACE7FFF7A6FBA9E7705D00F0C8F8B4
S113850000281ED0785D002805D1705D211C8022D2
S113851000F0AEF815E00021402200F07DFA0028BA
S11385200AD0211C705D402200F0A2F8211C021C1C
S1138530785D00F071FA04E0785D4021104A00F0A3
S113854081F8785D002809D08022211C00F090F881
S1138550021E03D0705D211C00F05EFA0135032D6C
S1138560CBD129B0F0BDC046E3F9FF1FAEEC00004B
S1138570BBEC0000C8F9FF1F00F9FF1FE4F8FF1F60
S11385807510000000FAFF1FE2EC000008B50A1C99
S11385900349031C0878191C00F03EFA08BDC046C4
S11385A0C8F9FF1F024B1A78024B1A707047C04675
S11385B0C8F9FF1FCCF8FF1F12230380004870473F
S11385C06BEC0000CF23038000487047F9EC0000F7
S11385D000B5031E052B0ED8094A80008058027886
S11385E0002A06D1032B08D1064B186803780B80A8
S11385F004E00A8002E0002000E0101C00BDC04638
S1138600C0EC0000FCF9FF1F13B5441E0548E4B29A
S113861000682301C318187B00941C680323A04737
S113862016BDC04608FAFF1F08B5044B18700001B8
S113863000F09AFB024B186008BDC04603FAFF1F06
S113864008FAFF1F37B5031C0D1C0020FF2B0CD0AC
S11386500648013BDBB2046819016418207B0093CF
S1138660111C24682A1C0223A0473EBD08FAFF1FE0
S113867013B5441E0548E4B200682301C318187BEF
S113868000941C680423A04716BDC04608FAFF1FC7
S113869013B50749421E0968D2B21301CB18187BDF
S11386A0002100921C680A1C0523A04716BDC04681
S11386B008FAFF1FF7B5038A041C0E1C4768151C33
S11386C09A4200D91D1CADB2002D28D0E3687A1956
S11386D062609A4215D3DB1B9BB22268E91A0093AD
S11386E053186360019102F08BFE002E12D0391CE6
S11386F0009A301C04F010FE009B2168F018019AC7
S113870006E002F07DFE002E04D0301C391C2A1C29
S113871004F002FE02F06CFE238A5B1B238202F04B
S11387206FFE281CFEBD0000F7B51D1C174E08ABDC
S11387301B78019131681B010093CB18171C5C68EE
S113874002F056FE052D09D0062D09D0042D16D1B0
S1138750201C01993A1CFFF7ADFF16E0258A11E0B1
S1138760012F03D13368009A9B189C68002C08D011
S11387702368258AA36063600023238202E0002526
S113878000E0251C02F03CFE281CFEBD08FAFF1F79
S1138790F7B5041C151C0F1C02F02AFE218A628AFC
S11387A0E38A88184019984202DD5D1AAD1AADB209
S11387B0A168AA18628201914A19E168A2602E1C7C
S11387C08A4205D3D31A2268A3609B1AEE1AB6B262
S11387D002F016FE0198391C321C04F09DFDB542CE
S11387E004D0B919AA1B206804F096FD02F000FE1B
S11387F0638AA28AAB4206D1238AEB189A18002313
S11388002282A38202E0AA18A2825B1B638202F086
S1138810F7FD281CFEBD000030B50A4B0A4A1B6850
S113882014780022A2420BD01D680132854204D183
S11388301D7B8D4201D1D0B203E0D2B21033F1E7F7
S1138840002030BD08FAFF1F03FAFF1FF0B5061C15
S113885085B0101C019102920393FFF7DDFF011E06
S113886001D000203AE0FFF7D7FF071EF9D01C4BD8
S1138870C5181C4B2D011B685D193388002B13D0C0
S1138880039800F071FA041C68600DD03388181C3A
S1138890009300F069FA0028E3D0009B2060606038
S11388A0A060C018E060E3827388002B11D00398A5
S11388B000F05AFA041CA8600BD07688301C00F033
S11388C053FA0028CDD020606060A0608019E06079
S11388D0E682029B381C2B60019B2B7305B0F0BD14
S11388E0FFFFFF0F08FAFF1F07B5032807D005286D
S11388F011D0002813D1101C00F0A8FE10E0138939
S113890001A80380002343801368064A19781823BA
S1138910FFF79CFF04E0101C01F07AFA00E000204D
S11389200EBDC04629870000F7B5041C019100293B
S113893036D1027843780D1C9A4261D102F058FD79
S1138940A178304B30481970FFF766FF2F49087043
S113895000280ED02E4A2F4B80181B6800011818CF
S1138960436820791A8A561D3618D88A864203DD50
S11389700D7002F045FD43E006321A82A11D8C42BF
S11389800CD09A68501C9860207810709868DA6847
S1138990904201D3186898600134F0E706252FE06F
S11389A01A4B1E78002E0DD102784378351C9A425A
S11389B026D187781448391CFFF72EFFFFB2061E14
S11389C006D11DE00F4A177800221A7002F018FD34
S11389D00F4A104BB6181B6836019E19E37870686D
S11389E0032B04D1C58A038AED1AADB208E0211C19
S11389F0019AFFF7CDFE0421051C78B200F058FB64
S1138A00281CFEBD04FAFF1F2987000005FAFF1F7A
S1138A10FFFFFF0F08FAFF1F08B5031E04D1081C4F
S1138A20111CFFF781FF05E00020FF2B02D0181C6A
S1138A30FFF7EAFD08BD07B5031C002083420AD0F6
S1138A406A461070507093701171012368460521B5
S1138A50D370FFF769FF0EBD38B5041C031C1A1B45
S1138A600133581E057892B2002DF8D1281C002A33
S1138A7003D0081C211CFFF7CFFF38BD08B5024BFB
S1138A801978FFF7E9FF08BDCCF8FF1FF0B50E1CFD
S1138A9085B0141CCB0604D52023137004239E43F5
S1138AA00134F30706D5002804DA2D232370474246
S1138AB0013400E0071C00230193022333402F4DAF
S1138AC00393002F2DD0BD4214D9281C0A2104F091
S1138AD0E5FE019B051C002B04D10128F3D1039B67
S1138AE0002B01D0302302E07307ECD52023237040
S1138AF00134E8E7002D01D001230193291C381C1F
S1138B0004F0CCFE631C0293031CC0B268433033F0
S1138B1023703F1A0A21281C04F0C0FE029C051C85
S1138B20CFE73027201C019B002D09D0002B09D052
S1138B30281C0A2104F0B2FE2770051C0134F1E759
S1138B40002B0DD1730703D52023601C237007E08D
S1138B50B30702D53023601C237030230370013027
S1138B60330704D50D2303700A23437002304023D6
S1138B701E4000D1067005B0F0BDC04600CA9A3B45
S1138B801FB56A46FFF782FF6846FFF777FF05B017
S1138B9000BDF7B5CB0602D52023137001324BB2CA
S1138BA0002B04DA3023137078235370023220230D
S1138BB00B40009308230B404026019307230E40EB
S1138BC019400F1C042900D90427FFB27F000F218C
S1138BD0141C3B1C8C46013BDBB2FF2B15D09D00C3
S1138BE0011CE9400D1C61460D40291C3031392916
S1138BF008D90099002902D0291C373102E0291C28
S1138C005731C9B221700134E5E7019BD019002B1B
S1138C1004D00D2303700A2343700230002E00D1C8
S1138C200670FEBD1FB56A46FFF7B3FF6846FFF73F
S1138C3025FF05B000BD10B5031C00229A56202A5A
S1138C4001D10133F9E700200F241A7851B22F29FA
S1138C500CDDD1B20A1C303AD2B200010133092A28
S1138C6002D90A1C573A22401043EEE710BD10B552
S1138C7000220378191C3039C9B2092906D9002BFE
S1138C8018D02D2B00D101220130F2E70023017806
S1138C900C1C303CE4B2092C07D85C00303CDB00EF
S1138CA0E31849B201305B18F1E7181C002A02D01E
S1138CB0584200E0181C10BD00B50378002B0FD0FB
S1138CC000228A565BB2934207D0D80FD1179A423A
S1138CD0484140420123184307E001300131ECE7E9
S1138CE000200856431E9841404200BD10B5031CA5
S1138CF00C78181C1C700A78013352B20131002A16
S1138D00F6D110BD00B5021C031C981A0133591E7C
S1138D10097849B20029F8D100BD00000E4B13B503
S1138D2000221A800D4B0E4A19600E4B14781960FC
S1138D301A1C0378A34203D0002B0CD00430F8E7AC
S1138D404388C9186B46116007335522994202D8EB
S1138D500A700131FAE713BD10FAFF1F0CFAFF1F66
S1138D60D2F8FF1F14FAFF1FF8B50E4F0E4E3B68E2
S1138D703488051C1C1903231C4201D09C43043471
S1138D800A4A631912689A420AD92A1C201C002133
S1138D9004F060FB3B68201CE31AED18358000E00A
S1138DA00020F8BD0CFAFF1F10FAFF1F14FAFF1F72
S1138DB0F8B50F4F0F4E3B683488051C1C194B1E29
S1138DC01C4202D04B421C4064180B4A63191268BF
S1138DD09A420AD92A1C201C002104F03BFB3B6860
S1138DE0201CE31AED18358000E00020F8BDC046D1
S1138DF00CFAFF1F10FAFF1F14FAFF1F054B00B5F2
S1138E001A68131C981A0133197880B25529F9D0BD
S1138E1000BDC04614FAFF1F034B1868034B1B68C0
S1138E20C01A80B27047C04614FAFF1F0CFAFF1F25
S1138E30044B1868044B1B68C01A044B1B88C01AE7
S1138E4080B2704714FAFF1F0CFAFF1F10FAFF1FBD
S1138E50F0B585B00392574F574A002313603B6027
S1138E60564B061C1B780C1C2578002D48D06DB27F
S1138E709D423ED1221CA31ADBB202930134002589
S1138E806557002DF7D1142058430430FFF76CFFC9
S1138E9002993860CB43E4182F1C6178002926D04E
S1138EA049B2331C01911A68002A1ED00021515680
S1138EB08C4601998C4516D15968026041601A8923
S1138EC00281002A01D00135EDB2598941819A8984
S1138ED082819B7BC373002901D1002A01D0013711
S1138EE0FFB2143001E01033DDE70134D5E701604F
S1138EF008E001340022A256002AFAD10134B3E773
S1138F002F1C02952B4C2368002B47D0002F2BD00D
S1138F100C207843043080B2FFF726FF264E284AFF
S1138F202368306094461A68002A19D05A89002AA6
S1138F3006D0624501D1002159815A89426003E07B
S1138F409989002901D0416001224168002901D09A
S1138F5001214172002A01D003600C301433E2E78E
S1138F600C235F43C01B3060039BE818C0B2FFF7BB
S1138F705BFB002D12D02468216800290ED02389C0
S1138F80002B09D003200121221CFFF7ADFCA073A4
S1138F90002801D1FF23A3731434EDE7094802F03C
S1138FA017FA094B00221A6002F024FE029805B059
S1138FB0F0BDC04618FAFF1F24FAFF1FD2F8FF1FA6
S1138FC0FFFF00001CFAFF1F20FAFF1F054A064896
S1138FD01188CB07DB17034049084B4098B2108037
S1138FE07047C0461CFAFF1F00B4FFFF184B37B58B
S1138FF01C682368002B29D0E27B0D231A4223D05E
S113900002F0F6F9A389002B02D1E37BD90716D429
S1139010237C002B0ED000256A46157055702168FC
S1139020281C0A7869468A700522CD700B71FFF7F7
S1139030F3FC2574E27B0A23134000D1E37302F0AE
S1139040DFF9201C626890471434D2E737BDC0466C
S113905018FAFF1F38B50C4B051C1C6802F0C8F940
S11390600D222368002B0CD0E17B114207D01B7822
S11390705BB2AB4203D002F0C3F9012002E0143426
S1139080EFE7181C38BDC04618FAFF1F00B5074BA0
S11390901B681A68002A07D0127852B2824201D1A2
S11390A0D87B02E01433F4E7802000BD18FAFF1FD8
S11390B038B5174B1C682368002B27D01B785BB28C
S11390C0834221D1002918D1124B1D68002D14D0E0
S11390D02B68002B11D09C420DD102F089F9A38991
S11390E0002B03D00C4A12689B186B600023E373B7
S11390F002F086F90AE00C35EAE74A0702D5E37B79
S11391001A0703D4E17301E01434D4E738BDC04630
S113911018FAFF1F24FAFF1F20FAFF1FF8B5194B96
S11391200E1C1C68171C002C2BD0174B1D682B68B9
S1139130002B26D01B785BB2834220D12368002BFE
S11391401FD09D4219D102F053F9EB7B02229343C5
S1139150EB732772002F04D1AE81002E04D1667206
S113916008E0002E00D10126084B1B68F6180123E5
S11391706660637202F044F903E00C34DEE71435F0
S1139180D5E7F8BD24FAFF1F18FAFF1F20FAFF1FC6
S113919038B5114B1D68002D1DD0104B1C68236879
S11391A0002B18D01B785BB2834212D12B68002BA2
S11391B011D09C420BD102F01BF900232B726B726D
S11391C0E37B02221343E37302F01AF903E00C3544
S11391D0ECE71434E3E738BD24FAFF1F18FAFF1F45
S11391E0144A154B11681B680131F0B5101C11604D
S11391F0002B1ED00224082504261A68002A18D041
S1139200597A002913D001685F68B9420FD1D17B24
S1139210214204D1294200D1D673197A117492895A
S1139220002A03D059688A185A6000E05A720C3335
S1139230E3E7F0BD20FAFF1F24FAFF1F37B5051C32
S113924033352B78002B11D0028B8A420ED86A4614
S1139250937001230024D370DD23147054701371B0
S1139260201C69460522FFF7D7FB2C7037BD000090
S1139270F0B50B1C34331A7801231A4085B0051C51
S11392800C1C9446002A05D00A8B0B8DD31A0B8331
S113929000230B85271C30373B78980711D0281CF6
S11392A01121DA0700D4132102F0C6FEC0B200284F
S11392B000D094E03B7803229343402213433B7055
S11392C08DE020201840029000D085E0268B002EEF
S11392D008D140229343281C3B7002F0C9FE201C95
S11392E0311C76E0E168E06A0A7840051AD504206A
S11392F0034202D083433B7014E0201C32300078D8
S11393000190824206D0201C31300078904209D16D
S1139310012E07D004221343221C30321370012380
S1139320019A02936046002833D062698B199A42ED
S113933004D8521A92B2002A51D000E0321CE38BB6
S11393405B089E420CD9B31A0293264BA800185806
S1139350029BC08C834203DB7608B24200D95208D8
S11393603B78402003433B70281C02F095FE061C0A
S1139370E06862698319E360934201D3A368E36000
S11393801848AD004359201CD98CFFF757FF268598
S113939025E0111C281C02F04FFE236840210133F4
S11393A02360231C30331A780A431A70029A002A65
S11393B015D1E36860690133E360834201D3A26895
S11393C0E260238BAD00013B2383064B201CEB584A
S11393D0D98CFFF733FF02E0281C02F049FE05B0E8
S11393E0F0BDC04634FAFF1FF7B51F1C08AB009050
S11393F00D1C141C1E7801F0FBFFB81E082800D9B0
S113940002E104F041FA09004C0072003F00D70069
S1139410010101010101B2007E4B36011B689E1956
S1139420E90401D5B66800E07668002C28D0E2078C
S113943003D5009802F0ACFE04E0A30702D500981F
S113944002F0F0FE610703D5009802F04DFE04E03F
S1139450220702D5009802F091FEF36AE10603D5D3
S113946080225201134303E0A20602D56A4A134044
S1139470F362630604D57F231D40331C33331D7010
S1139480B58DC2E0634B36011B68644A9E1973684C
S1139490DC6A144201D01D8CB7E01D8BB5E05D4B36
S11394A036011B689E19B668002D07D1F28B338BE9
S11394B0D31A9DB2A34200DBA7E0A5E001F0A0FF10
S11394C0301C291C221C0830FFF762F9051C01F02E
S11394D08FFF331C30331A7860231A4200D094E093
S11394E00098311CFFF7C4FE8FE04A4F36013968FB
S11394F001968B195E68291C301C0830221CFFF76A
S1139500D9F8331C34331B781A070CD5338CDC0799
S113951009D4F28BB3685208F1689A18914201D2C7
S1139520F26000E0F360F36A6022051C13426ED01F
S1139530321C303211781020014268D0348BA4469A
S1139540F48CA44563D88143117099065FD53E68B5
S1139550019C01203619B1680B1C30331A78024380
S11395601A700098FFF784FE51E02A4B36011B68FD
S11395709E19012C05D9023CB368A4B2002D10D168
S113958003E07368002D0CD107E0012C05D91D60A0
S11395905D6073681D605D6037E0A4000025E550E0
S11395A033E0A4001C190023E25CEA540133042BC9
S11395B0FAD129E0174D3601002C03D02B689E19EF
S11395C0B3681AE0296810248A195368191C3031C9
S11395D00878204211D0A04308709168CA6A9206A4
S11395E008D50B1C30331A78012002431A700098F6
S11395F0FFF73EFE2B689E1973689A6800251A616E
S1139600DA601D831D8400E0002501F0F9FE281CAA
S1139610FEBDC04608FAFF1FFFEFFFFF8080000079
S113962038B5051C3820FFF79FFB041E01D100202C
S11396300BE0281CFFF798FBA0600028F7D0431923
S11396402061E0606361E583201C38BDF7B5434EBB
S11396500091017A041C301CFFF7DEF8051C071C7E
S1139660002D03D00099490707D476E0291CFFF7A1
S1139670D3F8051C381C002D6FD0394A394BAF186C
S11396801B683F01DF19009B3E609B0707D5E088FC
S1139690267AFFF7C5FF3449B6008851B860009AAE
S11396A0324ED20706D5A088FFF7BAFF237A786036
S11396B09B00F050237A2C499B00CB58002B13D0ED
S11396C02268DA62237A627B9B00CB5834331A70A7
S11396D0237AE0889B00CB5864210093E37B5843B2
S11396E004F02AF9009BD884237A9B00F358002BBA
S11396F02CD0227B33331A70237AA188A07B9B0061
S1139700F358009148436421019304F015F9019A38
S113971064219084237AE07B9B00F3580193009B9F
S1139720584304F009F901992268C884237A9B00FC
S1139730F358DA62237A627B9B00F35834331A704D
S1139740237AA27A9B00F35832331A70237A211CAD
S11397503B73207A02F070FD281CFEBDE9930000E3
S1139760FFFFFF0F08FAFF1F34FAFF1F28FAFF1F3D
S1139770F7B5684A8B009C58674A80279D58E36A6E
S11397803F01061C01911F4014D0221C3032117875
S113979004200F1C0740BC4603D0814311700027EE
S11397A010E0271C32373F78B74202D101431170D1
S11397B0AFE067461A0605D5221C31321778BF1B65
S11397C07A4257412022134233D0132E23D12B1C2B
S11397D034331B78DF0714D5291C0831019802F0B3
S11397E081FC2A8B2B8DE968D31AAA68C318081A3E
S11397F02B83E860904202D2EB8BC018E860002310
S11398002B852B1C30331A7820210A431A706B687D
S113981001336B607DE0112E0BD12B1C3033197892
S1139820114276D0914319700198291CFFF720FD4D
S11398306FE0226801322260D9041AD52A8BEB8B9F
S11398409A420CD82A6916702B69696901332B6115
S11398508B4201D3AA682A612B8B01332B832B1CE7
S113986030331A7860231A4203D10198291CFFF778
S1139870FFFC238BE28B002F32D19A420BD90133A8
S1139880238323691E702369676901332361BB4203
S113989001D3A1682161E36A602213421BD0261C14
S11398A030363278D70616D4218BA28C914212D34B
S11398B0990609D52B1C30331A7802210A431A70F1
S11398C00198291CFFF7D4FC33781022134333701A
S11398D0636801336360114BE26A1A4211D018E0E5
S11398E0218C013121849A420BD9013323832369CA
S11398F01E702369676901332361BB4201D3A168E8
S1139900216133342078002803D040B20421FFF7CA
S1139910CFFBF7BD28FAFF1F34FAFF1F8080000039
S113992008B5034B8200D158FFF7A2FC08BDC0461E
S113993034FAFF1F10B5002808D08369981DC27F30
S1139940541C0C3252009B18C477998010BD10B57A
S1139950831CCC0706D504781480407800020443A5
S113996014800232981C8C0706D51C7814805B780E
S11399701B021C43148002324B0705D50378138065
S1139980417809020B43138010BD0000F7B5282469
S113999001935C43364B00901B6800201C19E38A3A
S11399A0089E834262D12283131C8A4200D90B1C75
S11399B0A28A9FB2E382974201D9628200E0638265
S11399C0F3680099658A1960B36880205A6829048D
S11399D01043284A114072680143116059684022BB
S11399E0514059609968E0684A409A60291CFFF721
S11399F0A1FF009A6260E28A638A9A4207D0E36810
S1139A00002B06D09B690633DB7F012B01D9E08A4A
S1139A102CE00198311C02F057F90028F7D17B1B88
S1139A209FB2009B5B190093A38A3D1C9F4200D9FF
S1139A301D1CF368009980201960B368ADB25A68A0
S1139A40290410430B4A114072680143116059689C
S1139A504022514059609968E0684A409A60291C44
S1139A60FFF768FF638AEB186382C4E7FEBDC04654
S1139A7044FAFF1F0000FF03F0B58BB01C1C10ABB1
S1139A8003900F1C161C1D7801F0B2FCA01E0428C4
S1139A9000D995E04D4B2D011B685D1903F0EAFEDA
S1139AA0031A67178500F80401D5AB6800E06B68FA
S1139AB0710608D59A69D11CC97FC80703D57F21CF
S1139AC00F400232D7779B690333DD7F79E06B68FF
S1139AD01D8A76E0AC68002C0CD1039805A902F02D
S1139AE0F3F8251C00286CD105A90091381C311C01
S1139AF0321C37E0A36900250333DB7FDA0760D526
S1139B00AF4206D1E28A238AD31AB34259DB9DB20B
S1139B1057E001F075FC391C321C201CFEF738FE9E
S1139B20061C051C01F064FCA36940270333DB7F9A
S1139B303B4246D1039805A902F0C6F8002840D15B
S1139B40A2696168E0680332431AD17F9BB20F4374
S1139B50D777321C9E4200D91A1C92B205AB6068BA
S1139B60111C0093039BFFF711FF051C29E06C688F
S1139B70391C321C201CFEF79DFDA3690427033306
S1139B80DB7F061C3B421FD001F032FCA369033388
S1139B90DA7FBA43DA77A169887E02F04DF90028AA
S1139BA0F9D001F02DFC301C0EE0002E01D0AB6882
S1139BB000E06B681A6800259A605A601D8200E014
S1139BC0002501F01DFC281C0BB0F0BD08FAFF1F96
S1139BD0F0B58BB06C4626340390201C049105929A
S1139BE01E1CFEF7EFFC039C01218C46624262417D
S1139BF0D2B2002307926F460578FA8C0195521B66
S1139C0092B2FA8402924278042A12D0052A23D00E
S1139C10022A42D14379039C1B1B5A425341DBB2B3
S1139C20002B02D1079D002D37D000270123BC460D
S1139C3033E0002B31D0049CFF2C02D08278A24266
S1139C402BD1059DFF2D03D0C2780323AA4224D132
S1139C50002E2CD0022320E0002B1ED0002E1CD07E
S1139C609D1E6A425541321C1168002912D0002DF4
S1139C700ED18F7884787C407F273C4208D14D797F
S1139C8009792D02294395888D4206D2918004E0FA
S1139C900832E9E7002D00D010600199029A4018BB
S1139CA0002AA8D1644660426041404230400BB073
S1139CB0F0BD37B58369051C0233DB7F002B13D05D
S1139CC0028A8A4210D86A46937001230024D37012
S1139CD0DD23137114705470201C69460522FEF7AD
S1139CE09BFEAB690233DC7737BD000070B5041C02
S1139CF080780B1C7F22011C114028254D430C4EFB
S1139D009043E27836681043627975192679120215
S1139D10324302F011F8E278EB1C002A01D111223F
S1139D2003E00435EA7F01210A43DA7770BDC046B7
S1139D3044FAFF1F38B5011C7F23194028244C43E3
S1139D400E4B00221B68FF201C19131CE56801F050
S1139D50F3FF0023E21CD377A21DE382D3779D4255
S1139D6003D02B822B68AB606B60A368002B04D0FC
S1139D7000221A821A689A605A6038BD44FAFF1F9A
S1139D8070B5041CC0B00D1C161C022806D11F4B54
S1139D90012218780023FFF71BFF34E08022684675
S1139DA00021520003F056FB002C02D0012C12D0EB
S1139DB028E0164B291C1878FF226B46FFF708FF92
S1139DC0083400AA1319083B1B68002B1AD0987892
S1139DD0FFF7B0FFF4E70D4B291C1878321C6B46D3
S1139DE0FFF7F6FE031C201C0024002B0BD00834C4
S1139DF000AA1319083B1868002803D00021FFF7B4
S1139E0075FFF4E7002040B070BDC04642FAFF1F62
S1139E10F7B5051C294F1C230430A97B284A3C684C
S1139E20FEF714FD0190AE7B2823002E0AD05E437A
S1139E30AB89A419A3826B89D90613D5231D2022CB
S1139E40DA770FE0687C01305843FEF78DFF082372
S1139E5083823860AA7C431C041CDA77301C291CDA
S1139E6002F024F8019B17495A18174B12011B687A
S1139E709A189368E360002B02D09C612B8923829B
S1139E80AB7BA376AB7B002B0CD0EB7B002B09D0F8
S1139E9028245C4339680C19A376A97B631DD97700
S1139EA0AB89A3825368A360002B03D09C61AA7C76
S1139EB0631CDA772D6801982560FEBD44FAFF1F04
S1139EC0799A0000FFFFFF0F08FAFF1FF0B5151C79
S1139ED01C4A85B0146828225043241827680E1C95
S1139EE0002F03D1A068002807D129E0081C1A1C00
S1139EF0291CB847072823D1F4E7631CD87F00281E
S1139F0003D040B20421FFF7D3F8A3680334E17F00
S1139F10A4460191019C04210C400120002C0FD186
S1139F20DA8A1F8AD21BAA4206DB181C311C2A1C9F
S1139F30FEF72EFC201C03E0019A63460A43DA77FD
S1139F4005B0F0BD44FAFF1FF0B58022C1B00E1C6D
S1139F5052000021051C684603F07CFA301CFF21E6
S1139F6000226B46FFF734FE002828D0154F00244A
S1139F706B461859002823D0002D0BD1002E03D195
S1139F808078FFF7D7FE18E000AA13199988FFF725
S1139F90ADFE12E082787F231340282253433A68AF
S1139FA0D31803330222D97F012D01D1A94302E042
S1139FB091430A1C01210A43DA770834D8E70120C7
S1139FC041B0F0BD44FAFF1FF0B58BB00D1C0492F4
S1139FD003930024062800D99CE203F055FC0A01EF
S1139FE072026B0207007A028B02920204982825FF
S1139FF04543B94B1B685D19EF8AEC68002F28D1E3
S113A000002C00D186E2238A002B1BD06268E16811
S113A0108A4202D3E08A121A62606068091A89B21D
S113A0200A1C994200D91A1C92B20399049B00910C
S113A030111CFFF7ABFCA269201C118AFFF739FE43
S113A040002467E2A26940200332D17F8143D177A3
S113A050F6E76B8ABB4200D290E0002C6FD0268AD0
S113A060002E6CD0A3699A1D988BD17F8446012958
S113A07001DDD88B98830139D177A2696146761ABC
S113A080131CB6B2059226820633DB7F591C4900A5
S113A0905B00D0184942002302911A1C0299023B2A
S113A0A08B4205D0C118898B8C46624492B2F5E785
S113A0B0964230D1002EBED1EB1CDA7F30231A42F7
S113A0C015D0A98A381C03F02DFC89B200290ED1C1
S113A0D0039A8821936852685868012601431160E5
S113A0E0596840225140596099684A409A606268B0
S113A0F0E368D71967609F4202D3E38AFF1A676057
S113A1000023EB829E4296D1059B40210333DA7FE4
S113A1108A43DA778FE76068E368C71967609F420C
S113A12002D3E18A7F1A67606068B61A1B1A99B273
S113A130B2B28E4200DB0A1C0023EB8275E7A98AC7
S113A140381C03F0EFFB89B2002914D12B8BBB42DE
S113A15003D1EB1CDB7F98060DD503998B684A6805
S113A1605868882101431160596840225140596060
S113A17099684A409A600024EC82CBE1FF1AAB8ACA
S113A180BFB23E1C9F4200D91E1CB6B2002C11D097
S113A190A3699A1DD17F988B012901DDDF8B9F83F1
S113A1A00139D177238AA2691B1A2382118A201CC0
S113A1B0FFF77FFD039869686A8AC3688A181A6082
S113A1C08368426859688020084344493704394009
S113A1D001431160986859684022514042405960D7
S113A1E09A60311C201CFFF7A5FB6B8AF6186E825F
S113A1F026E7394B0C781E6800278022F7829443A7
S113A200012C00D1A5E0022C00D1FEE0BC4200D01C
S113A21049E14878092800D991E003F02BFB8A90A2
S113A2209090904B05908550C8788A78CF798B7937
S113A230000210433F021F43FF22031C802193436B
S113A24089008B4216D008D880225200934228D12C
S113A25008AD281CFEF7B0F91FE0C02189008B422D
S113A26014D0C022D20093421BD1039B1C480093FC
S113A2700A2106E008AD281CFEF7A4F9039B2988EF
S113A28000933A1C0023FFF781FB43E108AD104023
S113A290291CFEF79DF900281BD0039A29880092F7
S113A2A0EFE733680424002B00D133E1039A681CE0
S113A2B0118A4CE08B780398032483742AE189780B
S113A2C0084C00202170FFF73FFE061E0CD000232F
S113A2D0237004241EE1C04644FAFF1F0000FF035C
S113A2E022EE000042FAFF1F8C4903240B6801335D
S113A2F0DB7F0393002B00D10CE16846A91C0122EB
S113A300263003F009F808AF039A7523FB70022383
S113A310BA703B71301CFE23391C07223E707E70DC
S113A3207B71FEF779FBF5E0039B7D4800930121E7
S113A33003E00398022100907A480A1CA2E73368DC
S113A3400424002B00D1E5E0039A281C118A002282
S113A35058E04B78881C04930A2B1DD00B2B02D099
S113A360002B46D135E06E4B04241B78002B00D122
S113A370D0E008AD03212A1CFFF7E9FAA978FF22EF
S113A380381CFFF7FDFCA9782A780120FFF7F8FCB8
S113A39043424341E41ABDE0614B04241B78002B83
S113A3A000D1B7E008AD02212A1CFFF7D0FA2978C2
S113A3B002203A1CFFF7E4FC002800D1AAE003992C
S113A3C00330009101210A1C3B1CFFF7DFFA3C1CFF
S113A3D0A0E0534B04241B78002B00D19AE0039A8D
S113A3E00221009250480A1C049BFFF7CFFA049CF8
S113A3F090E033680424002B00D18BE00398018A99
S113A400281C3A1C9847041C84E0497804910129CB
S113A41041D808AFA81C211C3A1CFFF798FA404BFE
S113A4201B78002B03D13B880424002B72D138887D
S113A4301F22282302405A430499B21803320823E6
S113A440012916D1D17F194200D1F9E59943336826
S113A450D177002B00D1F3E5C0B26C46E07701F070
S113A46005FC2E4A1F341368201C1B68002104229B
S113A470C8E7D27F134006D0039B022100932B48E8
S113A4800A1C002304E003980221009026480A1CB9
S113A490FFF77CFAD4E533680424002B3AD0281C57
S113A4A008210322AEE733680424002B32D0039A38
S113A4B0118AA5E7039B1A8A002A02D10498022371
S113A4C004E00398291C028A04980123FFF7FEFC88
S113A4D099E703998B7C002B07D0104B1F201B6836
S113A4E0CC2101331856FEF7A6FA0020011CFFF711
S113A4F02BFDA5E5094B1F201B68CB210133185602
S113A50005E0064B1F201B68CA2101331856FEF7CD
S113A51092FA95E5201C0BB0F0BDC04644FAFF1F2B
S113A52042FAFF1F40FAFF1F1EEE000020EE00005B
S113A53028235843034B1B6818180330C37F19435F
S113A540C177704744FAFF1F2822034B50431B680E
S113A55018180530C07F704744FAFF1F70B5041CFB
S113A56001200E1C151C02F033FF002807D102F055
S113A5702FFF002800D1412003235840C0B223B24A
S113A580002B05DA80235B421843C0B203235840F2
S113A5906404321C2B1C610C03F004F870BD03B27C
S113A5A070B5041C0E1C151C0120002B02DA640477
S113A5B0640C002002F00CFF002805D0211C321C82
S113A5C02B1C02F02DFF01E00120404270BD08B5B4
S113A5D0022804D003280ED0012817D10CE0002053
S113A5E002F0F6FE002811D080235B4218430021BC
S113A5F0C0B20A1C06E0002002F0EAFE002805D0E2
S113A60001210022131C02F0CDFF01E00120404291
S113A61008BD00B5402801DC303804E0602801DCC6
S113A620373800E03D3840B2C0B200BD08B500780C
S113A63040B2FFF7EEFF002800D00120FC23800287
S113A6401B02C01808BD000013B5042201A9041C94
S113A65002F0B6FE019B002B08D05A1C09D0064A12
S113A660141B9C4200D20194019803E08020C00096
S113A67000E0002016BDC046FB030100F8B5051C30
S113A6800E1C171C002809D0FFF7DEFF041DA40AC6
S113A6908023A402DB00E4182C1901E0FC2424022A
S113A6A00B4B9C4202D90020306010E0201CFFF7C5
S113A6B0CBFF3060002806D0201D391C012202F097
S113A6C07FFE201C03E08023DB00E418E8E7F8BDEC
S113A6D0FE03010008B501F067FE431E98414042A5
S113A6E008BD0000F0B587B00291141C494D00D19B
S113A6F08DE02E68002E2CD1471D4748FF210760AE
S113A7000822464802F0A6FE6A46301C05A9133208
S113A710FFF7B4FF061E53D0059A414BD118890A9E
S113A72089020591B74209D373189F4206D2301C9F
S113A730FFF7D0FF059BA34242D2FF186A46301CA4
S113A74005A91332FFF79AFF061E39D0B842E3D9A0
S113A75036E03148334900688219334853181118D8
S113A7600919890A9B0A89B29BB20191012918D956
S113A770301C012B4CD8822464020121A41A0191BB
S113A7800FE00133FC229F021202284EBF180393EC
S113A790B74215D8381CFFF757FF002805D1039896
S113A7A083B201998B42ECD10AE03B18B34202D93F
S113A7B082204002C01B011D381CFFF78BFFEEE70F
S113A7C02868022813D803231B1A261E9E4200D988
S113A7D01E1C124B05301818321C029902F09CFD05
S113A7E02A68A41BB3182B60029B9B190293002CAC
S113A7F002D1029800280AD107492A6808680299F8
S113A8008018221C02F084FE2B68E4182C6028684F
S113A81007B0F0BD48FAFF1F4CFAFF1F50FAFF1FA4
S113A820040400000004FFFFFF03FFFFFF03010017
S113A83073B5124A00241368051C0193201CA3421B
S113A8401BD00B780E4E1460211C221C281C337163
S113A85002F05EFE01A90422301C02F05DFD311CF1
S113A8600822281C02F054FE281C211C221C02F081
S113A8704FFEA04200D00194019876BD48FAFF1F14
S113A88050FAFF1F08B501F0DBF908BD08B56120D7
S113A890B721FEF7D0F808BDF8B53D4B3D4E1A6818
S113A8A0041C01321A6033780D1C0133DBB233709F
S113A8B03B2B4CD9384F3B780133DBB23B703B2BFD
S113A8C038D9364B1A780132D2B21A70172A24D9E1
S113A8D000221A70324A3348117803780131C9B220
S113A8E011700133DBB2062B01D9073BFAE7037081
S113A8F01D2907D12C4B1978022903D1012111708C
S113A90003221A702A0708D5E368002B05D000F04B
S113A9106FFDE268904700F073FDAB0608D56269ED
S113A920002A05D000F064FD6369984700F068FDD3
S113A93000233B70AA0708D56368002B05D000F0FC
S113A94057FD6268904700F05BFD00233370EB0510
S113A95008D5A268002A05D000F04AFDA3689847EC
S113A96000F04EFDAA0508D52368002B05D000F0A1
S113A9703FFD2268904700F043FD2369002B05D07A
S113A98000F036FD2369984700F03AFDF8BDC04653
S113A99058FAFF1F5DFAFF1F5EFAFF1F5CFAFF1FE4
S113A9A0CEF8FF1FCDF8FF1FCFF8FF1F0D4B1B780C
S113A9B0C3720D4B1B8883800C4B1B7883710C4B2B
S113A9C01B78C3710B4B1B7803720B4B1B784372C0
S113A9D00A4B1B7883720A4B1B6803618023037341
S113A9E07047C0465DFAFF1FD0F8FF1FCFF8FF1F66
S113A9F0CEF8FF1FCDF8FF1F5CFAFF1F5EFAFF1FA2
S113AA0058FAFF1FF7B5002801D1464B1960464D8F
S113AA10464C474F0A1C04230326AC46651EADB2C0
S113AA2035420CD162450FD9424D02335219DBB283
S113AA30062B02D80134A4B2F0E7073BF7E7BA4289
S113AA4006D80026019601E001270197002408E0BA
S113AA50394D01335219DBB2062BEBD9073BFAE728
S113AA600224019E002E0CD0012C0AD1334FBA428D
S113AA7017D9334C1D331219DBB2062BF0D9073B1F
S113AA80FAE7304E375D304E7E43B24209D9921B0D
S113AA90FB18DBB2062B01D9073BFAE70134E4B219
S113AAA0DFE70134E4B2284EA4460124B24209D9B6
S113AAB0264F0134D219E4B20133DBB2062BF5D9A7
S113AAC0073BFAE70026224FBA4204D9214F013648
S113AAD0D219F6B2F7E700273B2A03D901373C3AEB
S113AAE0FFB2F9E7D2B2019200280AD00372019BA7
S113AAF062468271C471C372877246728580016135
S113AB000FE0154962460A7014490C701449019CFF
S113AB100B70144B1C70144B1F70144B1E70144B91
S113AB201D80F7BD58FAFF1F0085E201B30700003E
S113AB308033E101007B1DFE80CC1EFE803B26009D
S113AB4080C4D9FF2CEE00008051010080AEFEFFCE
S113AB500F0E0000F0F1FFFFCFF8FF1FCEF8FF1F2C
S113AB60CDF8FF1F5DFAFF1F5EFAFF1F5CFAFF1F9F
S113AB70D0F8FF1FF0B58BB005AD01900C1C281C5C
S113AB800021142202F03AFF0199042910D10B2369
S113AB902B73002C0FD0281C01F020FC2A69002AFA
S113ABA009D1201C7B49FEF7A1F8001BC0B2EFE0DD
S113ABB0281CFFF7FBFE019B07261E403AD0002C01
S113ABC034D006261E40221C002E12D00021E87923
S113ABD0FDF75CFF2E270770421C0221A879FDF7C0
S113ABE055FF021C07700132A8880021FDF74EFFB3
S113ABF0021C01990523194219D0002E02D02023EA
S113AC00137001320221687AFDF740FF3A2606707C
S113AC10421C0221A87AFDF739FF021C067001329A
S113AC20E87A0221FDF732FF021C00E0221C141B0B
S113AC30E0B2ADE0002C00D19BE0019A102A0AD1C9
S113AC400023E3562B2B0BD101340023E356202B96
S113AC50FAD0012604E0019B302B01D1102101918F
S113AC60201CFEF704F8C2B2071C039223781A1CB6
S113AC70303AD2B2092A01D80134F7E7002102910F
S113AC808B4210D00134201CFDF7F1FFC0B20290BA
S113AC902378303BDBB2092B01D80134F8E7331CAD
S113ACA05A1E9341F6180022A25600239A4208D055
S113ACB00134201CFDF7DBFF321C511E8A4183B294
S113ACC0B618019A102A12D12278111C3039C9B24F
S113ACD0092901D80134F7E7211C202A07D14A7831
S113ACE00134303AD2B2092A01D830210191019AB3
S113ACF092060CD5029A0399AA71274AE971AB808E
S113AD00934232D8FA21C9005B18AB802DE0032EA0
S113AD1025D8301C02F0AEFD02080C15039A0299E6
S113AD206A72A972EB7220E02A69FFB2BF1806E0CA
S113AD303C23FFB25F432B690299FF187F182F61F0
S113AD400FE0E1221201FFB257432A690299BF18AA
S113AD503C224A43DBB2BF18FB182B6101E0002EF2
S113AD6003D0281C2969FFF74DFE019A302A00D12F
S113AD7074E7019B102B04D1084B059306232B7316
S113AD8002E0012205AB1A73281C01F027FB002006
S113AD900BB0F0BD38EE0000CF0700008DA8000016
S113ADA0F0B585B0039181880422029137490023CC
S113ADB00324029DA94214D24D1C214207D1344FD1
S113ADC00232DB19D2B2062A09D9073AFAE7314925
S113ADD001325B18D2B2062A01D9073AFAE7291CD4
S113ADE0E7E78779032421408C462B4D391C2B4EF1
S113ADF00197013900290AD001394C5D371C67439A
S113AE00A218DB19D2B2062AF4D9073AFAE7614646
S113AE1000290AD1019D022D07D9204F0132DB19E7
S113AE20D2B2062A01D9073AFAE7C679771ED219AF
S113AE30D2B2062A01D9073AFAE7457A847AC17A66
S113AE40E1200001684384463C206043604440188C
S113AE500090124847430098C719F818039B002B29
S113AE6011D00F4B029F1F800E4B019F1F700E4B82
S113AE701E700E4B1D700E4B1C700E4B19700E4B3A
S113AE801A700E4B186005B0F0BDC046B207000042
S113AE900085E2018033E1012CEE000080510100C5
S113AEA0D0F8FF1FCFF8FF1FCEF8FF1F5CFAFF1F7B
S113AEB05EFAFF1F5DFAFF1FCDF8FF1F58FAFF1F50
S113AEC010B586B0041C422301A80373019401F059
S113AED085FA021E012A05D1034B6B2032211C6026
S113AEE0FEF71CF906B010BD60FAFF1F30B50B4D1C
S113AEF0847B89B0201C69460522FDF7B9FB002834
S113AF000AD06A46D378002BF4D11379012BF1D1FE
S113AF102868FFF7D5FFEDE709B030BD60FAFF1FE1
S113AF20F8B5204B051C3221186802F0B7FC1E4905
S113AF30071C02F0B3FC2A1C0021041CFDF7A6FD2B
S113AF40194D44216C434170612181707921C17094
S113AF5073213D1B20220171E1210270861D427183
S113AF600901281C02F09AFC321C0021041CFDF784
S113AF708DFDE1231B015C433A262C1B471C067004
S113AF803C21201C02F08AFC3A1C0221051CFDF71E
S113AF907DFD0670421C3C2045430221601BFDF7E9
S113AFA075FDF8BD20FAFF1F8051010008B56C2023
S113AFB0FEF750F8002801D102F034F808BD7047BC
S113AFC070477047704770477047704770477047C5
S113AFD0F8B51A4D1A4F2B7839782022DBB2194C68
S113AFE0114210D12178194011420CD0164A174E43
S113AFF09078337802211840FEF7BAFB2B78DBB245
S113B000190700D532783A787F2A07D822783F2169
S113B0108A431A4202D00220FEF782FC227840239F
S113B0201A420AD02978194207D09A43054B1A705C
S113B030074B0422196891431960F8BD04C0064007
S113B04008C0064003C0064076FBFF1F07C0064049
S113B05024FBFF1FF8B51A4D1A4F2B78397820229C
S113B060DBB2194C114210D12178194011420CD095
S113B070164A174E5078337801211840FEF778FBB2
S113B0802B78DBB2190700D532783A787F2A07D8B3
S113B09022783F218A431A4202D00120FEF740FC65
S113B0A0227840231A420AD02978194207D09A43B9
S113B0B0054B1A70074B0222196891431960F8BDB9
S113B0C004B0064008B0064003B0064076FBFF1FFC
S113B0D007B0064024FBFF1FF8B51A4D1A4F2B7812
S113B0E039782022DBB21140184C0FD12078184057
S113B0F010420BD0164A174E107833781840FEF7DA
S113B10037FB2B78DBB2190700D532783A787F2ADF
S113B11007D822783F218A431A4202D00020FEF742
S113B120FFFB227840231A420AD02978194207D01B
S113B1309A43064B1A70084B01221968914319600F
S113B140F8BDC04604A006400BA0064003A006407C
S113B15076FBFF1F07A0064024FBFF1F38B58022A3
S113B1600A4B0B4C52049A6023680425AB4302201B
S113B1702360FEF7D5FB23682B4206D11D43054B04
S113B18025601A7840210A431A7038BD2081004096
S113B19024FBFF1F03C0064038B580220A4B0B4C2A
S113B1A052049A6023680225AB4301202360FEF712
S113B1B0B7FB23682B4206D11D43054B25601A7843
S113B1C040210A431A7038BD1081004024FBFF1F40
S113B1D003B0064038B580220A4B0B4C52049A60E7
S113B1E023680125AB4300202360FEF799FB236805
S113B1F02B4206D11D43054B25601A7840210A4392
S113B2001A7038BD0081004024FBFF1F03A00640D4
S113B210134A002310B513491360134B134C0B60EE
S113B22010211160124A1168124A1160124A1380E7
S113B230124A1368002B0AD0013B1360002B06D17D
S113B2402368DA0703D580229200134323600C4855
S113B2502168FFF721FB22680A4B1340236010BDCD
S113B26014D0034004D00340187C000020FBFF1FCF
S113B27000D00340F8170020F017002074FAFF1FD5
S113B28090FAFF1FFFFCFFFF30B5204A13789806A1
S113B29004D51F4B03201B78590636D41D4B0421BB
S113B2A01B6801200B4230D0194B47241D78022023
S113B2B025422AD01078840605D51C78072004403E
S113B2C0081C022C21D01178080705D5187807210D
S113B2D001400520032918D012780120910714D5C4
S113B2E01B7807221340042B0FD10B4B197803232F
S113B2F00B40834208D0002B04D00820032B04D039
S113B300012002E0062000E0101C30BD00E00740F0
S113B31001E0074010ED00E002E00740F7B5234AE2
S113B320234C1568236801905B1B1A1C511E8A412B
S113B33020489B1A5843642102F0B0FA1E4F1F4A5A
S113B340061C13883868834209D9802109024018F1
S113B350FA21C01A890002F0A1FA361A05E0FA218E
S113B360C01A890002F09AFA3618154B761926602D
S113B3703B6020680D490E4A086010480380114B59
S113B3801968002907D010490968196010688142BA
S113B39001D212681A60019A002A06D0216800209E
S113B3A0FFF730FB094B10221A60F7BDF817002095
S113B3B000D00340CD0C000004D00340F01700205F
S113B3C0187C000008D00340F417002014D0034078
S113B3D0054B10B51C682388002B00D1034B038058
S113B3E0FDF7F4FD208010BD90FBFF1F7B120000D1
S113B3F072B6024B1A6801321A6070471CFBFF1FB9
S113B400044A00B51368013B1360002B00D162B6F7
S113B41000BDC0461CFBFF1F08B5054B1A681A6027
S113B420FFF7E6FFFDF7DCFEFFF7EAFF08BDC046C5
S113B43000000440F7B5304E041C3368151C002B83
S113B4400FD12E4B01229343181C2D4A3C300190FE
S113B450D71A1888D853019802338342F9D101329C
S113B4603260284A1378274F5BB2002BFADA3A7815
S113B47030231A4200D03B70234B1C70092C0ED091
S113B48002D8062C0BD01BE0412C16D0432C17D12C
S113B4900A681E4B1A7028681D4B186010E01B4B7D
S113B4A00A0C1A701B4B0A0A1A701B4B1970062CD3
S113B4B006D1174B2A681A6002E00A68134B1A7007
S113B4C0FFF796FF33680F489847FFF799FF412C21
S113B4D00ED1124B1A78124B12061B781B0413431D
S113B4E00B4A127813430F4A1278120213432B604B
S113B4F0387831231840FEBD7CFBFF1FD4F8FF1FB2
S113B50034FBFF1F00000240070002400600024017
S113B5100800024005000240040002400B00024003
S113B5200A0002400900024010B5074B074C0022F4
S113B5301A60A368934205D0FFF75AFFA36898479F
S113B540FFF75EFF10BDC04608D0034090FAFF1F0E
S113B5500B4B37B51F221A600A4B1D68002D0DD006
S113B560094B01AC1B6823800023A3700123E37003
S113B570FFF73EFF201CA847FFF742FF37BDC04638
S113B58000B0034078FAFF1F10B0034010B5094B18
S113B590094A1B781B019B18802252049A60074BAE
S113B5A01C68002C05D0FFF723FF0020A047FFF7FD
S113B5B027FF10BDB4FAFF1F0081004084FBFF1F6A
S113B5C010B5094B094A1B781B019B1880225204B1
S113B5D09A60074B1C68002C04D0FFF709FFA047B2
S113B5E0FFF70EFF10BDC04618FBFF1F008100408F
S113B5F064FAFF1F0268802310B51A421CD0144A53
S113B6004C00A25AD40403D51205120D026013E0B3
S113B6100360012906D0022909D000290CD10D4B61
S113B6200D4A06E00B4B0D4A1C68224003E0094B0F
S113B6300B4A186802401A600A4B8900CC58002C47
S113B64004D0FFF7D5FEA047FFF7DAFE10BDC046D1
S113B65070FBFF1F3C800440FFFFFFFEFFFFFFFD68
S113B660FFFFFFFB28FBFF1F08B502480221FFF77D
S113B670C1FF08BD00A0034008B502480121FFF73F
S113B680B9FF08BD0090034008B502480021FFF748
S113B690B1FF08BD00800340F7B5047801900E1C8B
S113B6A0E4B20125002C22D02C421CD0AC430F2E36
S113B6B00DDD331C103B01229A40012A04D0202ABC
S113B6C007D1FFF731FF04E0FFF7A6FE01E0019A7E
S113B6D01570074AB3009F58002F04D0FFF788FE67
S113B6E0B847FFF78DFE6D000136EDB2DAE7F7BD1E
S113B6F0B8FAFF1F08B506480021FFF7CDFF05483B
S113B7000821FFF7C9FF04481021FFF7C5FF08BD52
S113B71005C0074006C0074007C007400E490301A3
S113B7205B18002210B59A60041C6400FFF760FEE9
S113B7300A4A0323A3401C1C1378A343137007D1A4
S113B740074A084B022111601968074A0A401A6027
S113B750FFF756FE10BDC0460071034079FBFF1F82
S113B760007003403C800440FFFF7FFF08B5174B87
S113B770032299680A40032A11D10122DA60144B8A
S113B78018780223184007D0FFF732FE114B1B68CC
S113B7909847FFF735FE02E0FFF7C0FFF4E70E4BD2
S113B7A0032299680A40032A0ED10120D860084B6D
S113B7B01B781A0701D4FFF7B1FFFFF719FE054BF9
S113B7C05B689847FFF71CFE08BDC0460071034044
S113B7D079FBFF1F88FBFF1F10710340F7B50E1C98
S113B7E00090171C1D1CFFF703FE00980C23584300
S113B7F02C4B2D4C196801900A18A26092685306CC
S113B80002D42B1C103301E02B1C18336360043367
S113B810E360301C7968009A231CFEF7D5FB061EF2
S113B820032E06D0042815D0012828D1FFF7E8FDFF
S113B83036E0A3686168586880221043086058683D
S113B84040214840586098684140996039680A43EB
S113B8503A6022E0009A002A04D184232B61AB6170
S113B860101C09E00098FEF76FFE104B1A684301A4
S113B870D31884221A619A610821FEF759FE094BF4
S113B88001981A680A4B1218916820680B40034308
S113B89080211943236039601360FFF7B1FD00264E
S113B8A0301CFEBD68FAFF1F7CFAFF1FACFAFF1FB5
S113B8B00800FF03F7B5A14FA14D3B782C781C403D
S113B8C000D13AE10823201C984300D18FE0FFF710
S113B8D08FFD012004424BD098499A4A33230B70C0
S113B8E013780226334313702B7830218B432B704B
S113B8F0954B196840238F689F4300230B608F602A
S113B9001178B1431170914A91491370914A0870AA
S113B91013709148914A1370137003709048037028
S113B92090480370904803709048037090480370E7
S113B93090480370904803701370904A1370904AB3
S113B9401370904A137004230E781E40FCD18E4B62
S113B9508E4A1B688E4F9A608E4A04201A60311CEE
S113B960321C3B1CFEF730FB794B0D22BE741A705F
S113B970A00717D5884B1A78510705D5874A874FF2
S113B9805268019201327A601A78900705D583498A
S113B990824F09680A1C01323A60062267481A700D
S113B9A002230370E1060CD5644A302313702B780C
S113B9B02022134300212B7005200A1C0B1CFEF7C8
S113B9C003FB20231C420BD05C4F30223A702A78B0
S113B9D000219A432A7006200A1C0B1CFEF7F4FA75
S113B9E0FFF70EFD0823201C5449984308700820D3
S113B9F0044200D15FE76A4A634B1478196824094A
S113BA0016786301CB18624D06421FD00C226243A4
S113BA104D4909688A18AA609268570604D41A1C0A
S113BA2010326A60143303E01A1C18326A601C3343
S113BA30EB60FFF7DDFC221C2B1C00210320FEF72A
S113BA40C3FAFFF7DDFCAA7C404B69E010780422BE
S113BA5010401A1C002801D00832402028601068C9
S113BA608601B60D2E823C263040042802D03428AC
S113BA7025D057E00C256543334E802730684119A3
S113BA808868000701D509680F403148A1000918EA
S113BA900978C80602D5201C012101E0201C0221DE
S113BAA0FFF79CFE33685D198023002F03D02968BB
S113BAB099430B1C01E02A6813432B6039E02F687B
S113BAC000200C26186198611F4D364866437F0696
S113BAD008D42F68BE19B6683040C02608603043C9
S113BAE0886007E02F68BE19B6683040C0268860B9
S113BAF0304308600C266643286881194820486052
S113BB00201C0021FFF76AFE012805D02B689E192E
S113BB10316880230B4333600A4B20211A788A430F
S113BB201A7006E084221A619A61201C0821FEF72B
S113BB30FFFC024A08231370BDE6F7BD80200740CE
S113BB40842007409420074068FAFF1F982007408C
S113BB50C0200740C4200740D0200740C820074029
S113BB60D4200740D8200740DC200740E0200740CD
S113BB70E4200740E8200740EC200740F420074079
S113BB80F8200740FC200740ACFAFF1F880008009B
S113BB907CFAFF1FC8000800882007406CFAFF1FCA
S113BBA0902007400800FF030E4B10B51B6884006B
S113BBB04033E2500C4A89018318C9B21970C31783
S113BBC0DB0E1B18094A5B119B009B18084A1040A6
S113BBD004D5202201385242104301300122824010
S113BBE01A6010BD08ED00E000E400E000E100E0B0
S113BBF01F00008038B50D4B01251A680C4C2A43F0
S113BC001A60802323600B4B05221A601C20032139
S113BC10094AFFF7C9FF2368402213432360074BF7
S113BC2013221A6023681D43256038BD3880044000
S113BC30000004400400044019B40000080004405B
S113BC40074B00B51A680C231A4204D0054B552241
S113BC501A60AA221A60044B20221A6000BDC04652
S113BC6000810440048104408CF00F40134B021CFB
S113BC70196880239A43530140B210B5CB180028A9
S113BC8013DA0F48910009180C2042430D4800684C
S113BC908218546840208443546000221A619A61D7
S113BCA00B78022293430B7006E01968986804220B
S113BCB0914390431960986010BDC046ACFAFF1FD1
S113BCC0C020074068FAFF1F38B5184A0C1C1849F1
S113BCD01568820052181278031C0120510723D5DD
S113BCE00C225A4313495B010968ED188A18A260B3
S113BCF0FFF77EFBA3689B685A0604D42B1C103301
S113BD006360143503E02B1C183363601C356368CF
S113BD10E5601C6880231C4003D0FFF771FB022000
S113BD2002E0FFF76DFB201C38BDC046ACFAFF1FD4
S113BD30C020074068FAFF1FF0B59C46394B3A4EC5
S113BD401C688B0085B09E194B01151CE4180191E9
S113BD500296364A364BFF2812D100213170A16178
S113BD602161A1602160019C0C20604312681218BB
S113BD70916011601A78302082431A7031704EE05D
S113BD801978102631431970029E80233178061CDD
S113BD909E4303960C231268012E06D1019E0027B0
S113BDA07343D3185F60242607E0019E482773433A
S113BDB00126D31808225A600E4340B2002825DB1E
S113BDC0606800280CD12B1C654500D263469DB2E7
S113BDD0281CFCF7C9FF6060281CFCF7C5FFE06065
S113BDE008231E43134B2D041D4080232F431A1C8C
S113BDF03A43A260402297433B4323600B4B019C90
S113BE001A680C236343D3189F6001E004231E4384
S113BE10039C002C01D010231E43029C267005B005
S113BE20F0BDC046ACFAFF1FC020074068FAFF1FF0
S113BE30842007400000FF03F7B50C26184B464347
S113BE40184F1C6839684301E4188B5940252B426C
S113BE5002D00022009201E0083400952268802577
S113BE60131C2B40019301990123002916D192013F
S113BE70920D6168FEF72AF8022301280ED03B6870
S113BE8000999E19B268084B13400B432A1C1A43AD
S113BE902260326815402B433360019B181CFEBDA1
S113BEA0ACFAFF1F68FAFF1F0800FF03F7B5484A02
S113BEB04B7C10680C1C474901330140802000066C
S113BEC001431160227CDBB2012A05D1424AA02140
S113BED01068C902014308E0404A802110688901C2
S113BEE001431160E0213E4AC90011603D4A8021AE
S113BEF01068C902014311601D1C102B00D91025C4
S113BF00EDB20C206843FCF72FFF374E374B3060FF
S113BF10197880220A431A7034490B785BB2002BDB
S113BF20FADB334F022380213B7068019940FCF710
S113BF303FFF304D304B2860000A18706A882F4B41
S113BF401A70EA782E4B1A702E4A002313702E4A68
S113BF503B7013700423117819400191FBD1082020
S113BF602F68FCF701FF786008202F68FCF7FCFEBF
S113BF702B68264AF8609A60254A18201A603368AC
S113BF80244A03219A60204B0D221A70224BED2281
S113BF901A70224BFF221A70214BBF221A70214AB9
S113BFA0FFF702FE019A204B11481A701F4B8B2297
S113BFB01A701F4B06221A700123037062891A42F9
S113BFC005D00A4940230B701A4B10221A70F7BD92
S113BFD000700440FFFFFFBF048004403880044029
S113BFE068D004403480044068FAFF1F0C210740E5
S113BFF094200740ACFAFF1F9C200740B020074064
S113C000B420074098200740C0200740880008005B
S113C010C8000800080008001020074080200740DE
S113C02088200740B5B8000000210740842007405D
S113C0308C2007400821074010B50B4B8200D358D1
S113C04001221C7964B2002C0CDA084C824020686E
S113C050024322601A79D9718022D97852420A4364
S113C060DA700022101C10BD78EF000024FBFF1FC3
S113C070084B820000B5D358002801D1DA7A00E0D9
S113C0801A7A7F2A05D8D9787F220A4040210A43A8
S113C090DA7000BD78EF00000E4B70B58400E458F0
S113C0A00D4B0E4D1B5C40261B015B192579E57871
S113C0B0B543E5709A600124196009498440201C45
S113C0C00C6820430860D8688021C9050143D96001
S113C0D0101C70BD78EF0000B4EF00000081004038
S113C0E024FBFF1F002070471C4B820010B5011C6D
S113C0F0D45801281ED000280ED0022829D1184B6C
S113C10080221868520102431A60C022154B920023
S113C1101A600E20144A1AE0114B80221968D200CA
S113C1200A431A60C022114B92001A600C200221AB
S113C1300F4A0CE00A4B8022196812010A431A6064
S113C140C0220C4B92001A600B4A0D200221FFF70B
S113C1502BFDE37808221343E37010BD78EF000051
S113C160388004400CC00440D1AF000044A0044017
S113C170D9B0000010B0044055B00000034B80005B
S113C180C3583722D9780A40DA70704778EF000034
S113C1901C4B820010B5011CD45801281ED0002865
S113C1A00ED0022829D1184B80221868520102436C
S113C1B01A60C022154B92001A600E20144A1AE02D
S113C1C0114B80221968D2000A431A60C022114B15
S113C1D092001A600C2002210F4A0CE00A4B8022C4
S113C1E0196812010A431A60C0220C4B92001A60AB
S113C1F00B4A0D200221FFF7D7FCE37824221343D6
S113C200E37010BD78EF00003880044008C004409B
S113C210D1AF000040A00440D9B000000CB00440ED
S113C22055B00000034B8000C3582421DA788A43B8
S113C230DA70704778EF0000F8B54D4B8200051CAA
S113C240D45801281AD0002808D0022800D08EE043
S113C250484B80201F684001384314E0454B802040
S113C2601E68C00030431860434B44481F6838437D
S113C2701860CB7A0B2B0DD99D230EE03D4B80200B
S113C2801E68000130431860CB7A0B2B6DD85B001D
S113C2903B4801E03B485B001B5AD804C00EDBB2AC
S113C2A0207063700B68384E0620DF070AD57F279D
S113C2B07755184010D0580701D5032300E0022316
S113C2C0A3700AE0FF277755184005D05E0701D513
S113C2D01323F5E71223F3E7A070002D06D00F68AF
S113C2E0FF0603D523782020034323704B7BD80714
S113C2F030D5264B26495E5D802337017F185B04C9
S113C300BB60E31D7B60234B022118680143196065
S113C310214B301C595D214B9A58FFF745FCE278BC
S113C3203F231A408023E2705B42002D03D1E27A5E
S113C3301343E37204E0217A194313432172E37037
S113C340174B6D00FB60EB1C80256D421D43154BA4
S113C350F5540CE07F23002D03D1E27A1340E372FD
S113C36005E0227A1340237201E04E2395E7F8BDDD
S113C37078EF00003480044004800440000001048D
S113C38098EE00009CEF000076FBFF1FB4EF000066
S113C390008100403C80044084EF000088EF0000EE
S113C3A0800052A00010024038B5840A4518A40247
S113C3B00920211C0022FFF73DF8002806D1802324
S113C3C02A1BDB009A4202D9E418F1E7012038BDA8
S113C3D008B58021C900FFF7E7FF08BD70B5041C4C
S113C3E0007BF023984301380A2800D9C8E001F003
S113C3F041FA08063D3639ACB9272B312400002315
S113C4002EE0604B80221868920502431A605E4B4E
S113C41000201860227B1E1C5C4D910605D5216905
S113C420FEF7F0FA23692B6004E0201C0121FEF7DB
S113C430B7FC286010233360A2E0554B19680AE06A
S113C440201CFEF7B3FA9BE0201C0021FEF7A8FC99
S113C450206195E02169201CFEF7D4FA90E00123C5
S113C460013300E000230133013300E000230133F2
S113C470217B484A7F2905D91568012199408D43BC
S113C48015607DE03F4980200E68800530433E4DB5
S113C49008602968C80703D53C4800212960016069
S113C4A026683D4998004650002129601068012102
S113C4B0994001431160394E022B16D1334A384B4F
S113C4C010681968884201D912681A601968304ADC
S113C4D0142011601A68334B03211A60324AFFF7A3
S113C4E063FB32680423134305E0152003212F4A1C
S113C4F0FFF75AFB10233360237B5E0622D52C4BB7
S113C500C0221868120302431A602A4B2A4A187878
S113C5107D23984303D11188284B994209D0284997
S113C52000230B6027490B801E490B60264B1380A8
S113C53001E0FEF7F3FE254B254A1968914201D824
S113C540244A1A6010232B601AE0124B04221D683F
S113C550201C954300211D60FEF722FC104B18603F
S113C560002381E7637AE12212015A43A37A3C2132
S113C5704B43D218E37AD218174B1A60002377E79B
S113C580002070BD3C80044014D0034000D0034020
S113C59008D0034020FBFF1F90FAFF1F1CD003406C
S113C5A0A8FAFF1FF417002029B5000011B20000FB
S113C5B00070044000F00740F217002035CA000064
S113C5C0F8170020F017002035CAFFFF04D00340FD
S113C5D0177C0000187C000074FAFF1F0C4B30B568
S113C5E0C0180003002A03DA0A4B03241A4000E0AF
S113C5F0094C0123E443002909D0194204D00568F9
S113C600994325401543056004305B00F3E730BDD2
S113C610490004008BF8FF7F77070000F0B5071C82
S113C620007985B00138082801D900F0F9FC01F03F
S113C6302BF9800145009A00F9024002F704F7043F
S113C640F7040900B97BBC68FF2920D1CF4DD0493C
S113C6502B78A3432B703A7ACE4B1A700022012315
S113C660002C09D0B868184203D03E6888180664C4
S113C6709C435B000432F3E7C74A79790720FFF74C
S113C68093FABA682B7813432B7000F0C9FCBB896A
S113C69018221A40083A002692B20296102A02D8AA
S113C6A0BE48805C0290980701D500F08BFC042200
S113C6B01A4001D000F088FC00F02AFC387B0128E5
S113C6C001D900F0ADFC0E217B5E002B03DAFFF7ED
S113C6D025F800F0A5FCB24B3A688000C250FEF782
S113C6E087FEB04B3A7B032519785200281C9040F2
S113C6F08143F88928409040021C0A431A70FEF7CF
S113C7007FFE3C7BA84B2401E418A84B80221E68C2
S113C710120432431A603868A54B00221A60904212
S113C72005D079791620A34AFFF73EFA00E00125E7
S113C730FB890522134201D00022A260B9680122BC
S113C7402160E2601A0703D53A7B8023043204E0B7
S113C750DE0605D53A7B902304321A43964B1A60C1
S113C760A56000F05DFC954BA02118787A7901430F
S113C7701970934B80211868890408431860930941
S113C780012B5AD0002B03D0022B78D000F048FCA8
S113C790864B802118684904014319607879C023C5
S113C7A09843072801D900F03BFC864B01F062F85E
S113C7B0040D163A1F28313A186880218900014374
S113C7C01960D0218900804B34E0186880218900E9
S113C7D001431960D02189007C4B2BE0186880212B
S113C7E0890101431960D0218900794B22E018683E
S113C7F08021890101431960D0218900754B19E01A
S113C800186880214901014319608821C900724BCD
S113C81010E018688021890001431960D021890043
S113C8206E4B07E018688021890001431960D0210C
S113C8306B4B890019606B4B43E05C4B1C682143D4
S113C84019607B79C0218B430DD0012B01D000F0FE
S113C850E7FB5C4B80211868890001431960D021F3
S113C8608900614B08E0574B802118688900014317
S113C8701960D0215D4B890019605D4B21E04B4B61
S113C88080211E68C904314319607B79C0218B4320
S113C8900CD0012B00D0C3E34A4B80211868C90097
S113C8A001431960D0218900524B08E0454B802197
S113C8B01868C90001431960D0214F4B89001960E1
S113C8C04E4B3F210A40191C0831C020C867B97A71
S113C8D0C8060FD54A4980200C6840049040844320
S113C8E00C60384980200C6880002043086045486B
S113C8F045490860B97A01327F2903D9D100591812
S113C900242002E0D100591828204860B87A3989D7
S113C910860604D549089960F988490802E0013976
S113C9209960F988D2009A189160B97A3F220A4036
S113C93084E12249A0200C78BB7B2043BA680870AC
S113C9401F4980200C68800404430C60012B13D021
S113C950002B02D0022B63D062E30C21785E1349D2
S113C960002801DA294B0DE00C68802040042043A4
S113C97008601C4C112661E00C217C5E0B49002CE4
S113C98048DA234B0A6813400B6049E304C00740AC
S113C990B8FAFF1F07C00740F5B60000B9EE000063
S113C9A088FBFF1F79FBFF1F007103403C8004409C
S113C9B0007003406DB7000018800440005006402A
S113C9C004800440388004400C90044010900440DB
S113C9D074D004407CD0044014C00440049004404B
S113C9E018900440008003402490044020900440A8
S113C9F0009003400CA0044048A0044000A0034061
S113CA000C8004400304000048900440FFFFFFFE34
S113CA10FFFFFFFD0C68122620430860884C0DE0E0
S113CA200C21785E8749002801DA874BAAE70C6855
S113CA308020C0042043854C086013260021216017
S113CA4025680296280600D52160211CC0250831DE
S113CA50CD677F4D0021AA4205D9072902D00131B3
S113CA605208F8E77A4A7B4E89B25D000191A953D6
S113CA70B889C00604D58021480101990143A9530E
S113CA80A26075493A689B005A50002A08D0734A3C
S113CA9079799A580298FFF787F8735BC82201E006
S113CAA0735B882213437353735B1B051B0D236055
S113CAB0B6E2B968090608D5BB7D002B00D0AFE209
S113CAC0604B1C68620052081A60BD7D002D00D0C6
S113CAD0A6E25C4E802330681B0603433360BB68C8
S113CAE0D90706D59D07ED0FAD015A0701D42022C1
S113CAF015431C0702D5B98A594A1180C0229200F5
S113CB00134200D186E0574B0022DA77FC7D564869
S113CB102401802324185B04A360C823DB03E3609F
S113CB20524BF968A3604E4B21603A686360504BE6
S113CB30A360002A0FD0E3684E490B43E360BB7D3A
S113CB404D4998004250F87D4C4AD05479794C4A6A
S113CB50FFF72AF851E03B698022920093423DD0CE
S113CB6014D8402B33D007D8102B2CD0202B00D036
S113CB7056E2E26880232CE0802B2CD080225200E5
S113CB80934200D04CE2E268A0232CE080225201C0
S113CB9093422AD00BD88022D200934221D0802203
S113CBA01201934200D03BE2E268802322E080221B
S113CBB0920193421CD08022D201934200D02FE2F2
S113CBC0E268B02316E08023E2685B0113E0E268C8
S113CBD0C0239B010FE0E268802304E0E268C023E5
S113CBE001E0E268E023DB0105E0E268902301E074
S113CBF0E268A0231B021343E36032680223134359
S113CC003360FA7D1F4BA821D154E268C123DB05B0
S113CC101343E360BB685C0601D580231D431A4BB4
S113CC20DD77FDE1BB68BD79FA7C9E0130D5002A31
S113CC3000D0F5E1034B154A186802401A60EFE191
S113CC40009003403C800440FFFFFFFB00A0034032
S113CC50FFFF000070FBFF1F28FBFF1FCCEE00004E
S113CC6000F0034003F003400081004000FE0F0188
S113CC7000FE0F008000008064FAFF1F18FBFF1FF6
S113CC80C1B500000010024002F00340FFFFFFF7AF
S113CC90002A00D0C4E1990200D524E11A025BD530
S113CCA0CA4B80221C68120522431A60B968C84A1C
S113CCB0CBB29360B87C07230340CE0001D510208B
S113CCC00343D360080A0123034001901362CB029B
S113CCD033D5BF4B87245C6280201468BC4BA446C8
S113CCE0664680240642F8D0986C8446D86C844406
S113CCF0586C061C186C66443618D86B3618986B3A
S113CD0036187608B446604626023043D862986ED8
S113CD108446D86E8444586E8444186E8444D86D16
S113CD208444986D84446046400806431E635E6AEA
S113CD30A6435E621E68A6431E6001984123184004
S113CD401062B87CA24B4006400F50620A0103D522
S113CD505A6A08210A435A62BB685C0200D4C2E0E2
S113CD605E0108D5032D04D92A1C1A3AD2B2032A2B
S113CD7001D820221543964E58040CD57A7D002BF9
S113CD8008DA032A04D9111C1A39C9B2032901D8B3
S113CD9020210A437260190100D5A3E0C021C9050E
S113CDA03A680B4200D190E0336A04210B437C1DA6
S113CDB033620194E47F87488C40802324185B0409
S113CDC0A360B0239B03E360834BF969A360834BA7
S113CDD02360834B6160A360002A10D0E36881491B
S113CDE00B43E360FB7C804998004250019AD07F5A
S113CDF07E4AD05479797E4AFEF7D6FE51E03B6AEA
S113CE008022920093423DD015D8402B33D008D8CD
S113CE10102B2CD0202B00D002E1E3681A43E260EF
S113CE203FE0802B2BD080225200934200D0F7E0C9
S113CE30E268A0232BE080225201934229D00AD831
S113CE408022D200934220D080221201934200D04B
S113CE50E6E0E26823E08022920193421CD0802223
S113CE60D201934200D0DBE0E268B02316E08023D5
S113CE70E2685B0013E0C023E2689B000FE0E26815
S113CE80802304E0E268C02301E0E268E023DB00E1
S113CE9005E0E268902301E0E268A0231B0113434C
S113CEA0E3604A4B02221868019902431A60FB7C32
S113CEB0CA7F80212833494219434E4BD154E2683A
S113CEC0C123DB051343E3600CE0002A0AD0F97C9C
S113CED0494B8900CA5079790F20484AFEF764FE0D
S113CEE040231D433560B968CA0100D498E0BA698B
S113CEF0002A00D194E0364B8C0206D419684E0601
S113CF0003D4802118680842FCD01B69138087E091
S113CF10D80515D5042900D982E039488026B60001
S113CF2005688E40311C29430160802149000B4271
S113CF3002D0520052080A43B87B211CFFF74EFB73
S113CF40012500260196002C6AD0B868284235D005
S113CF50BB7B019E5B012B489B191E5CFF2E2CD0D2
S113CF600323321C1A40520027490392F2088918FD
S113CF70264AB608B61803988C46191C33788140A3
S113CF808B433370BB7B01991E4A5B015B189B5C2E
S113CF901F483A6899000A5007200340012199402C
S113CFA0CBB261460B701B4A7979FEF7FDFD039BFA
S113CFB0029A9A40337813433370AC43019E6D0058
S113CFC00136BFE7144AA5E7144AA3E73C800440AE
S113CFD000B003400081004000FE0F0110B0034088
S113CFE000FE0F008000008084FBFF1FB4FAFF1FC7
S113CFF08DB500000010024078FAFF1F51B5000003
S113D00038800440D8EE000005C0074000C0074047
S113D010B8FAFF1FF5B6000003000080020000808C
S113D02005B0F0BDF7B5694C0423256800951D4291
S113D03040D0674A1268002A03D022689A43131C1E
S113D04037E064490A6850050ED5634A40261078D3
S113D05030431070614807783E4306701278D50754
S113D06002D522689A432260086800050FD55C4BFC
S113D07040201A7802431A705A4A167830431070C6
S113D0801B78DA0703D523680422934323600B68D3
S113D090DD040FD5544B40211A780A431A70534AC1
S113D0A01078014311701B78D80703D52368042234
S113D0B0934323604E4E35780195FEF7E5F8042836
S113D0C031DD4C4B1B6898002DD54B490B68DA06B3
S113D0D029D54A480268002A25D000230B60484B12
S113D0E01F68D71B012F1CD9FA26013FB6007E43C7
S113D0F01D68F70BAC46BC44944502D01A68BF18AF
S113D1000760404A1568AE1B7604760C16603E4AEA
S113D11016801A6803689A4203D9394B1A68374B48
S113D1201A6010230B6030BFFEF7AEF804280CDD44
S113D130304B1B68980008D52F4B1A68D10604D5CC
S113D14000221A600120FEF7E9F823685A070BD47D
S113D150009D204B25601A68500523D51F4A4020A6
S113D1601178814311701DE0284B1A7828231A4244
S113D170EED0274B27221A70264B582226481A70C5
S113D18020220178244B1142FBD04022197811420D
S113D190FCD01749019D0D700C211A780A400C2A05
S113D1A0FBD1D5E71868000504D50E4A4020117854
S113D1B0814311701B68D90404D50C4B40211A78A3
S113D1C08A431A70FEF71CF9F7BDC04610ED00E063
S113D1D024FBFF1F3480044005A0064000A0064045
S113D1E005B0064000B0064005C0064000C0064039
S113D1F0004006403C80044014D0034008D0034063
S113D20000D0034004D00340F017002000E00740A2
S113D21004400640054006400640064008B56C2020
S113D220FBF734FF0923021C00201A4201D0FEF749
S113D2302BF808BDE02208B5031C9043082853D8F6
S113D24000F018FB05080B0D1C232F3740006C2041
S113D25000214BE00022274B0AE000221BE0264B72
S113D26020211A780A431A70224BC02219780A43E3
S113D2701A70224B04211A688A4334E01E4B202181
S113D2801A780A431A70822205E01B4B08211A7887
S113D2900A431A700322174B04211A70174B1A6899
S113D2A020E0154A02201178014311701F22934394
S113D2B011E0114A02201178014311701F22934397
S113D2C0012207E00C4A02201178014311701F2249
S113D2D09343032213430A4A1370064B04221A7021
S113D2E0064B19680A431A606C200121FBF7E0FE23
S113D2F008BDC04601E0074000E0074010ED00E033
S113D30002E00740024A034B00B51A60FEE7C0463C
S113D3100400FA050CED00E0F7B50E2A01D800234D
S113D3203FE0234CE368002BF9D1051C8218032746
S113D330531B0326394204D00B7801312B7001357D
S113D340F6E780277F040193194AA760354208D085
S113D3500126354201D0174E01E0B343164ED66084
S113D36002E0164FB343D7601A02120A21606560C7
S113D370A260E668802252023243E260019AED180C
S113D380C918D31A80225204A6681642FCD000227F
S113D3909A4203D08E5CAE540132F9E70023E36075
S113D3A005E0934203D0CC5CC4540133F9E7FEBDDD
S113D3B03081004080005A0080006C0080004800EA
S113D3C008B5031C081C191CFFF7A6FF08BD0000C4
S113D3D037B5F421051C0902684608226B425D41F9
S113D3E0FFF79AFF0D4C009B6D422543A34202D1E7
S113D3F0019BAB420FD0F821684609020822FFF7CF
S113D4008BFF009B0020A34206D10198401B45429C
S113D4106841400000E001203EBDC04655555555C9
S113D42070B5022801D0F42400E0F8242402083462
S113D4308900D5186418101CADB283B29D4207D080
S113D440461C211C0122FFF767FF0434301CF4E75B
S113D450002070BDF7B584180E2A01D8031C30E0F3
S113D4601B4BDA68002AF9D10D040A022A430A4345
S113D4700D062A4301920325021CA61A2A4202D051
S113D48011700132F9E7134F134C80256D049D6030
S113D4903440DF602F1C27439F6001AF1F600F4F94
S113D4A058609C601419DF609219944202D0217074
S113D4B00134FAE79A682A42FCD0054B0022DA606C
S113D4C004E0A34202D019700133FAE7FEBDC0465E
S113D4D03081004080000800FCFFFF00800009004C
S113D4E008B5002809D001280AD001300BD1002149
S113D4F008220648FFF7AEFF05E0044B186803E076
S113D500024B586800E0002008BDC0466CFAFF1FBB
S113D510F7B503230191161C204C002909D1226878
S113D5201A4201D1002038E09A432260042200927A
S113D53004E0021C9A43184022600090009B0425DA
S113D540ED1AB54200D9351C154A009B0199D7182C
S113D550381C2A1CFFF7E0FE019A114B52197F195F
S113D56004330192761B9F4210D3062021680C4A93
S113D570FDF760FF051E0FD1236809480433FF211E
S113D58004222360FFF766FF009502E023685D191B
S113D5902560002ED2D1C5E70120FEBD80FBFF1F10
S113D5A0B0FAFF1FF0B585B00193002643B20F1CFB
S113D5B0151CB34202DA7F2318400126420608D51F
S113D5C0F4200002FEF704FFF8200002FEF700FF3B
S113D5D002E0F824022800D0F424019B2402002B4A
S113D5E008D0019A231C0833BF00DF19AB189BB283
S113D5F0019311E0002E09D0F4200002844201D1ED
S113D600F8200002FEF7E4FE002615E0201CFEF7D9
S113D610DFFE002F10D030E0019AABB29A420BD05B
S113D6202B78174A381C134303A9042203930437A5
S113D630FFF76EFF0135EFE703A8211C0422FFF773
S113D6406BFE104D039BAB4205D0201C03A90422A2
S113D6500395FFF75DFF002E0FD10434042203A8C5
S113D660211CFFF759FE039AAA4206D0054B201C41
S113D67003A904220393FFF74BFF002005B0F0BD7C
S113D68000FFFFFF5555555510B5124A124913486E
S113D690891A00238B4203D0C45CD4540133F9E7C4
S113D6A00F49104A914205D10F4A10490023891AA3
S113D6B0181C08E00E480023801A8342F4D0CC5C86
S113D6C0D4540133F9E78B4203D0D41820700133CA
S113D6D0F9E710BDC0F8FF1FE0F8FF1F28F00000B5
S113D6E09060000090600000E0F8FF1F94FBFF1FB3
S113D6F00EDA00003D4B80221968D2000A4310B5AF
S113D7001A603B4B03211A688A431A60394A3A4B20
S113D7101A603A4B1A6802231A40394B00D00C2283
S113D7201A60384B08221A70374BA4221A70374BF0
S113D730A022374C1A7002211A1C2078344B08425C
S113D740FBD0102118780842FCD10C201978014034
S113D7500829FBD12F49272008702F495820087029
S113D760202118780842FCD0402118780842FCD0C7
S113D7702A492B480860282111700C211A780A4084
S113D7800C2AFBD1274B284A28491360284ADA601F
S113D790284A1A61284A5A61284A9A61284A1A630F
S113D7A0284A9A60284A9A63284ADA62284B294A06
S113D7B01A608B4201D00433FAE7FFF765FFFF21BB
S113D7C004222548FFF746FEF8F762FE234A244B5D
S113D7D0244825491A60FBF7A1FA244824490A225F
S113D7E0FBF736FBFBF702FCFCE7C046388004403D
S113D7F054F00F400301030080A0044050F00F4098
S113D8000081044002D00740014006400040064029
S113D810064006400440064005400640448004405B
S113D8200000011000F8FF1F08ED00E0BCF8FF1F26
S113D830BFAF0000C1AF0000C3AF0000C5AF000020
S113D840C7AF0000C9AF0000CBAF0000CDAF0000F0
S113D85040F8FF1FCFAF0000B0FAFF1FFC170020F5
S113D86090FBFF1F94EF000094FBFF1FB8EF000034
S113D870B0EE000002B4714649084900095C490051
S113D8808E4402BC7047C04603B471464908400048
S113D8904900095A49008E4403BC7047002934D01A
S113D8A00123002210B488422CD301242407A1426E
S113D8B004D2814202D209011B01F8E7E400A1422B
S113D8C004D2814202D249005B00F8E7884201D3C6
S113D8D0401A1A434C08A04202D3001B5C0822439E
S113D8E08C08A04202D3001B9C082243CC08A0420F
S113D8F002D3001BDC082243002803D01B0901D0FB
S113D9000909E3E7101C10BC7047002801D000206F
S113D910C04307B4024802A14018029003BDC046A8
S113D920D90000000029F0D003B5FFF7B9FF0EBC01
S113D9304243891A1847C046002941D010B4041C38
S113D9404C40A44601230022002900D54942002866
S113D95000D5404288422CD301242407A14204D29A
S113D960814202D209011B01F8E7E400A14204D27A
S113D970814202D249005B00F8E7884201D3401A91
S113D9801A434C08A04202D3001B5C0822438C08B3
S113D990A04202D3001B9C082243CC08A04202D31D
S113D9A0001BDC082243002803D01B0901D009090D
S113D9B0E3E7101C6446002C00D5404210BC7047BD
S113D9C0002806D003DB0020C043400801E080208B
S113D9D0000607B4024802A14018029003BDC046E5
S113D9E0190000000029EBD003B5FFF7A7FF0EBC18
S113D9F04243891A1847C0467047C04600B5031C05
S111DA008218934202D019700133FAE700BD78
S113DA10436F6E6E656374696F6E2074696D6564BF
S113DA20206F75740D0A00001B00780020000000B0
S113DA3017005D600A0000000041444D494E00207B
S113DA4020755461736B6572264B494E4554495396
S113DA50000000000000000000000000000050145E
S113DA6003030000000000000D0A0A48656C6C6F97
S113DA702C20776F726C642E2E2E204B494E455409
S113DA8049530D0A0052544320416C61726D206663
S113DA90697265640D0A00574F4B454E202D2000D6
S113DAA0676F696E6720746F204C53532061676100
S113DAB0696E0D0A00726573746F72696E67205720
S113DAC0414954206D6F64650D0A00436F6D6D61AB
S113DAD06E64206C696E6520626C6F636B65640DA7
S113DAE00A00000020E6000023E600000012000007
S113DAF033E6000038E600000200000057616B6561
S113DB007570000020E6000023E60000001200000B
S113DB1033E6000038E60000020000003F3F3F000B
S113DB200820080057616B65757020726573657411
S113DB300000000020E6000023E6000000120000C0
S113DB406BEA000074EA00000500000089EA0000A6
S113DB5092EA000005010000AAEA0000B3EA00000E
S113DB6005020000C7EA0000CFEA00000503000038
S113DB70EAEA0000F3EA00000504000013EB0000E9
S113DB8022EB0000051500003DEB00004BEB00000C
S113DB90051600001DE7000068EB000005110000F9
S113DBA03CE7000041E7000003060000E5E6000052
S113DBB0CFE600000000000033E6000038E6000075
S113DBC00200000031000000312E35003200000058
S113DBD07065726970686572616C206661696C75E4
S113DBE07265004A5441470020E6000023E6000025
S113DBF000120000EAE60000F2E60000010A00005C
S113DC0006E700000DE7000001010000E5E6000062
S113DC10CFE600000000000033E6000038E6000014
S113DC2002000000536F667477617265004C6F6385
S113DC306B75700045787465726E616C00436C6F2F
S113DC40636B206C6F73730020E6000023E6000012
S113DC500012000033E6000038E600000200000075
S113DC6074616D706572000068E1000082EB000071
S113DC70000400009AEB00009CEB0000000500008B
S113DC8072E10000B7EB000000060000C6EB0000E4
S113DC90C8EB000000070000E2EB0000E4EB00002A
S113DCA00009000003EC000005EC0000000A00007D
S113DCB051E4000014EC0000000E000053E40000E6
S113DCC023EC0000000F00003EEC000040EC0000DC
S113DCD0001000005BEC000013E6000000110000DF
S113DCE0E5E60000CFE600000000000033E6000097
S113DCF038E600000200000020E6000023E60000F1
S113DD00001200001DE7000029E7000006020000E1
S113DD103CE7000041E70000030600005DE7000067
S113DD2064E70000030700007CE7000084E70000CC
S113DD30030200009DE70000A7E70000060A0000B8
S113DD40B9E70000C2E7000006090000D4E70000BC
S113DD50DDE7000006080000F1E70000FCE7000032
S113DD60060C00000EE8000018E80000060B000096
S113DD7032E800003CE80000060D000049E800001D
S113DD8051E80000011F000071E8000078E800007D
S113DD900120000094E800009AE80000010000005F
S113DDA0A7E80000B0E80000011A0000E5E6000062
S113DDB0CFE600000000000033E6000038E6000073
S113DDC00200000020E6000023E60000001200002C
S113DDD033E6000038E6000002000000486F737468
S113DDE020646562756767657200000020E60000C4
S113DDF023E60000001200004BE6000056E6000097
S113DE00051C000066E6000072E60000051D000027
S113DE1085E6000090E6000008000000B6E6000079
S113DE20BFE6000008010000E5E60000CFE60000C0
S113DE300000000033E6000038E6000002000000A5
S113DE4068DC00000F0C00006CE5000028DF000017
S113DE50140200007BE5000034DB0000160C000017
S113DE608EE5000058DF00000F0F0000A0E5000061
S113DE70F8DC000011110000B3E50000E8DB00004D
S113DE8011050000C2E50000ECDD00000D070000F4
S113DE90D1E50000C4DD00000D020000DEE5000055
S113DEA004DB00000D020000EBE5000048DC00008C
S113DEB00F020000FCE50000E4DA00000F0200009D
S113DEC010E60000556E646572766F6C7461676568
S113DED000333030000000003630300000000031E4
S113DEE0323030000000323430300000003438303A
S113DEF03000000039363030000000313434303026
S113DF000000313932303000003338343030000012
S113DF10353736303000003131353230300032336D
S113DF20303430300000000020E6000023E600001A
S113DF300012000033E6000038E600000200000092
S113DF404F444400004556454E004E4F4E45005048
S113DF506F7765722D6F6E0020E6000023E60000E7
S113DF6000120000BCE80000BFE80000010F000040
S113DF70ECE80000EFE80000011000001BE90000DD
S113DF801EE90000011100004EE9000051E9000003
S113DF90011B000069E900006CE90000011C00009D
S113DFA083E9000086E90000011D00001AE7000073
S113DFB09BE90000011E0000BDE90000C5E9000066
S113DFC001020000E3E90000EBE90000010B00009E
S113DFD005EA00000FEA00000104000026EA000040
S113DFE031EA0000010500003CE700004EEA0000B1
S113DFF0010C0000E5E60000CFE600000000000090
S113E00033E6000038E60000020000004E4F4E45A3
S113E010000000005254530000000000584F4E000E
S113E02000000000455A504F525400536F667477F5
S113E0306172652076657273696F6E20000A0A0D3D
S113E040000A0D3D3D3D3D3D3D3D3D3D3D3D3D3D9C
S113E0503D3D3D3D3D3D0A0D000D0A4241442046F3
S113E0604F524D4154202D207175697474696E6747
S113E0700D0A000D0A424144204C454E47544820A5
S113E0802D207175697474696E670D0A007A0044F5
S113E0906F776E6C6F6164696E672E2E002A000DB7
S113E0A00A5465726D696E617465642C20726573BF
S113E0B0657474696E672E2E2E000A0D536572699D
S113E0C0616C206E756D6265723A200044657669F4
S113E0D06365206964656E74696669636174696FF8
S113E0E06E3A20004E657720616C61726D20736515
S113E0F0740D0A00416C61726D20636C6561726518
S113E100640D0A004E65772074696D65207365742B
S113E1100D0A004E65772064617465207365740D83
S113E1200A0030203D2052554E0031203D205741F9
S113E13049540032203D2053544F500033203D2099
S113E140564C50520034203D20564C50530035203C
S113E1503D204C4C530036203D20564C4C5330004F
S113E16037203D20564C4C53310038203D20564C2E
S113E1704C533300205B6163746976655D004C61C8
S113E1807374207265736574206361757365203DD3
S113E19020000A0D53797374656D206D656D6F727F
S113E1A079207573653A0A0D0046726565206865C5
S113E1B06170203D20002066726F6D20000A0D55AD
S113E1C06E7573656420737461636B203D20000D6C
S113E1D00A54686520646576696365206861732004
S113E1E06265656E206F7065726174696E67206622
S113E1F06F72200042616420706F7274206E756DBE
S113E2006265720D0A000D0A506F7274206469729F
S113E210656374696F6E3A20004F55545055540D20
S113E2200A00494E5055540D0A00496E76616C69D6
S113E2306420706F72740D0A00506F7274206973D9
S113E24020696E7075740D0A00506F7274207374B7
S113E2506174653A2000310D0A00300D0A000D0A80
S113E2603F3F0D0A23004D656D6F72792044697339
S113E270706C61790D0A00202020200046696C6CC6
S113E2800D0A0057726974650D0A00457261736561
S113E290640D0A004572617365206661696C65648A
S113E2A0210D0A00436F6E6E656374696E672055B5
S113E2B053422077697468205253323332202D2020
S113E2C0646973636F6E6E65637420555342207482
S113E2D06F20717569742E2E2E0D0A00506C6561C5
S113E2E07365207573652055534220636F6E6E65A8
S113E2F06374696F6E21210D0A00506C656173654A
S113E30020737461727420646F776E6C6F61643A09
S113E310000A0D427965204279650A0D000A0D5004
S113E3206172616D65746572207365740A0D000A0B
S113E3300D54656D702E20506172616D6574657247
S113E340207365740A0D000A0D506172616D657465
S113E35065722076616C7565203D20000A0D4E6F54
S113E3602076616C696420706172616D6574657298
S113E3707320617661696C61626C650A0D000A0D37
S113E3804F726967696E616C20706172616D65744A
S113E39065727320726573746F7265640A0D000A86
S113E3A00D466163746F727920706172616D65747A
S113E3B065727320726573746F7265640A0D000A66
S113E3C00D506172616D657465727320696E76615A
S113E3D06C6964617465640A0D000A0D4E657720EA
S113E3E0506172616D65746572732076616C6964E5
S113E3F0617465640A0D000A0D436F6E6669677582
S113E400726174696F6E2073617665640A0D0049E8
S113E4106E636F72726563742064617461206C65ED
S113E4206E6774680D0A000D0A53657269616C2089
S113E430636F6E66696775726174696F6E0D0A0049
S113E44042617564203D2000696E76616C696421C7
S113E450003700380020426974730D0A0020737479
S113E4606F70206269742873290D0A00466C6F77F7
S113E47020636F6E74726F6C200048696768207740
S113E480617465722000250D0A004C6F7720776156
S113E4907465722000555342204572726F72204396
S113E4A06F756E746572730D0A002D204352432DEF
S113E4B03136206572726F72733A002D20435243D5
S113E4C02D35206572726F7273203A0055534220C5
S113E4D04572726F7220436F756E74657273207229
S113E4E0657365740D0A00656E61626C650064692C
S113E4F07361626C65000D0A496E76616C69642013
S113E5007377697463680D0A00496E636F7272658C
S113E51063742073657269616C2073706565640D42
S113E5200A00496E636F7272656374207061726968
S113E53074790D0A00496E636F7272656374207397
S113E540746F7020626974730D0A00496E636F7290
S113E5507265637420666C6F7720636F6E74726F7C
S113E5606C0D0A000A0D0D004D41430020202020AF
S113E570204D61696E206D656E7500204C414E2002
S113E580636F6E66696775726174696F6E002020CF
S113E5902053657269616C20636F6E6669672E0033
S113E5A020496E7075742F4F7574707574206D6585
S113E5B06E750020202041646D696E2E206D656E9D
S113E5C0750020202053746174732E206D656E7560
S113E5D00020202020555342206D656E75002020B8
S113E5E02020493243206D656E75002020446973F4
S113E5F06B20696E74657266616365004654502FC2
S113E60054454C4E455420636F6D6D616E647300C8
S113E61020202043414E20636F6D6D616E64730052
S113E620757000676F20746F206D61696E206D6571
S113E6306E750071756974004C6561766520636F51
S113E6406D6D616E64206D6F6465007573625F65E6
S113E65072726F72730053686F772055534220654E
S113E66072726F7273007573625F636E745F72733C
S113E670740052657365742055534220636F756E40
S113E68074657273007573622D73657269616C00D1
S113E69052533233323C2D3E555342206D6F6465E4
S113E6A02028646973636F6E6E65637420746F20D1
S113E6B07175697429007573622D6C6F61640055FE
S113E6C053422D535720646F776E6C6F616400441E
S113E6D06973706C6179206D656E75207370656304
S113E6E0696669632068656C700075705F74696D34
S113E6F0650053686F77206F7065726174696E6727
S113E7002074696D65006D656D6F72790053686F73
S113E71077206D656D6F7279207573650073686F0E
S113E720775F636F6E6669670053686F7720636F06
S113E7306E66696775726174696F6E007361766580
S113E740005361766520636F6E66696775726174E4
S113E750696F6E20746F20464C4153480072656A9D
S113E760656374005265736574206E6F6E2D7361FA
S113E770766564206368616E67657300726573749F
S113E7806F726500526573746F726520666163749D
S113E7906F72792073657474696E67730073686F40
S113E7A0775F74696D6500446973706C6179206486
S113E7B06174652F74696D65007365745F74696D48
S113E7C065005365742074696D652068683A6D6DE1
S113E7D03A7373007365745F6461746500536574A0
S113E7E020446174652064643A6D6D3A797979796D
S113E7F00073686F775F616C61726D004469737058
S113E8006C617920616C61726D20642F7400736592
S113E810745F616C61726D0053657420616C617228
S113E8206D20286461746529282B295B74696D65E2
S113E8305D0064656C5F616C61726D0044656C655C
S113E840746520616C61726D0073686F775F6C70C2
S113E8500053686F77206C6F7720706F7765722034
S113E8606D6F646520616E64206F7074696F6E7380
S113E870007365745F6C70005B6F7074696F6E5DBC
S113E88020536574206C6F7720706F776572206DEC
S113E8906F646500726573657400526573657420F6
S113E8A0646576696365006C6173745F7273740088
S113E8B05265736574206361757365006D64004D02
S113E8C0656D6F727920446973706C6179205B6146
S113E8D06464726573735D205B3C6C3E7C3C773E84
S113E8E07C3C623E5D205B6E756D5D006D6D004D20
S113E8F0656D6F7279204D6F64696679205B616420
S113E90064726573735D205B3C6C3E7C3C773E7C3B
S113E9103C623E5D205B76616C5D006D66004D651A
S113E9206D6F72792046696C6C205B6164647265FA
S113E93073735D205B3C6C3E7C3C773E7C3C623E6A
S113E9405D205B76616C5D205B6E756D5D0073644C
S113E9500053746F7261676520446973706C6179E8
S113E960207B6173206D647D00736D0053746F723E
S113E970616765204D6F64696679207B6173206DE2
S113E9806D7D0073660053746F726167652046691C
S113E9906C6C207B6173206D667D0053746F7261B3
S113E9A06765204572617365205B61646472657399
S113E9B0735D205B6C656E2D6865785D00736574AE
S113E9C05F6464720053657420706F72742074798C
S113E9D07065205B312E2E345D205B3C693E7C3CAF
S113E9E06F3E006765745F646472004765742064F9
S113E9F061746120646972656374696F6E205B3150
S113EA002E2E345D00726561645F706F7274005203
S113EA1065616420706F727420696E707574205B18
S113EA20312E2E345D0077726974655F706F727475
S113EA300053657420706F7274206F7574707574F0
S113EA40205B312E2E345D205B302F315D0053610D
S113EA50766520706F72742073657474696E6720B4
S113EA6061732064656661756C74007365745F62BC
S113EA70617564005365742073657269616C20620A
S113EA806175642072617465007365745F73746F7B
S113EA9070005365742073746F70206269747320FE
S113EAA028312F312E352F3229007365745F626946
S113EAB074730053657420646174612062697473B3
S113EAC02028372F3829007365745F7061720053F2
S113EAD065742070617269747920284556454E2FFB
S113EAE04F44442F4E4F4E4529007365745F666C46
S113EAF06F770053657420666C6F7720636F6E7454
S113EB00726F6C2028584F4E2F5254532F4E4F4E35
S113EB104529007365745F686967685F7761746528
S113EB20720053657420666C6F77207374616C6C2B
S113EB3020282529205B312E2E39395D0073657418
S113EB405F6C6F775F7761746572005365742066DC
S113EB506C6F772072657374617274202825292084
S113EB605B312E2E39395D0053686F7720736572DF
S113EB7069616C20636F6E66696775726174696F31
S113EB806E00436F6E666967757265204C414E2056
S113EB90696E74657266616365003200436F6E6608
S113EBA069677572652073657269616C20696E743A
S113EBB065726661636500476F20746F20492F4F4B
S113EBC0206D656E75003400476F20746F2061649A
S113EBD06D696E697374726174696F6E206D656EB0
S113EBE075003500476F20746F206F766572766903
S113EBF065772F73746174697374696373206D65C9
S113EC006E75003600476F20746F20555342206D97
S113EC10656E7500476F20746F20493243206D651F
S113EC206E7500476F20746F2075744641542064DC
S113EC3069736B20696E746572666163650039007F
S113EC404654502F54454C4E455420636C69656EB0
S113EC507420636F6D6D616E647300610057444F7F
S113EC60470056312E342E3030380012010002EFA6
S113EC70020108A21544000001010203010803492E
S113EC80006E0074005553422052657365740A0D7A
S113EC90005553422053757370656E6465640A0DA4
S113ECA00055534220526573756D650A0D00456E1B
S113ECB0756D657261746564202800290A0D000071
S113ECC0CBED0000D8EC00000EEE0000C8ED000013
S113ECD004EE00007DEC00000A034D0061006E00AC
S113ECE07500436F6D6D616E64206C696E652062A2
S113ECF06C6F636B65640D0A000902CF00060104A2
S113ED00C000080B00020200000009040000010218
S113ED100200050524000002052401010004240268
S113ED200205240600010705820340000A090401C4
S113ED3000020A00000507050102400000070581E2
S113ED4002400000080B0202020000000904020055
S113ED50010202000505240000020524010100044B
S113ED6024020205240600010705840340000A0961
S113ED70040300020A00000507050302400000071F
S113ED80058302400000080B04020200000009048D
S113ED90040001020200050524000002052401010B
S113EDA0000424020205240600010705860340002E
S113EDB00A09040500020A000005070505024000CF
S113EDC00007058502400000000102040309040055
S113EDD02C01000058020000B0040000600900008B
S113EDE0C01200008025000040380000004B0000E5
S113EDF00096000000E1000000C20100008403004E
S113EE0090D003000A0343006F006E0066001003F5
S113EE104D0079002000500072006F006400000073
S113EE2001000A0600020000004001001F1C1F1E12
S113EE301F1E1F1F1E1F1E1F4E6F20616C61726DEF
S113EE4020656E61626C65640048544D004A504709
S113EE500047494600435353004A530042494E0079
S113EE6054585400424D500049434F003F3F3F0027
S113EE7057646F6700617070006D61696E74656ED0
S113EE8061636500757362006B6565706572006C23
S113EE906F77506F776572008813C409E2047102BA
S113EEA039019C0068004E0027001A000D0007007D
S113EEB0015775616D6B6C000001000000000000DB
S113EEC000020000000000000003000089B60000FA
S113EED079B6000069B60000FFFFFFFFFFFFFFFFE8
S113EEE0FFFFFFFFFFFFFFFFFFFFFFFFFFFFFFFF2E
S113EEF0FFFFFFFFFFFFFFFF05FFFFFFFFFFFFFF18
S113EF00FFFFFFFFFFFFFFFFFFFFFFFFFFFFFFFF0D
S113EF10FFFFFFFFFFFFFFFFFF06FF0708090AFFD0
S113EF20FFFFFFFFFFFFFFFFFFFFFFFFFFFFFFFFED
S113EF30FFFFFFFFFFFFFFFFFFFFFFFF0EFF0FFFBE
S113EF40FFFFFFFFFFFFFFFFFFFFFFFFFFFFFFFFCD
S113EF50FFFFFFFFFFFFFFFFFFFFFFFFFFFFFFFFBD
S113EF60FFFFFFFFFFFFFFFFFFFFFFFFFFFFFFFFAD
S113EF70FFFFFFFFFFFFFFFF00A0064000B00640B9
S113EF8000C0064002020200D5B1000099B10000A1
S113EF905DB1000001000014000000001127891376
S113EFA0C509E30472023901D1009D004F00350008
S113EFB01B000E000001020070EE000085A8000096
S113EFC0000000000A00010075EE00006962000004
S113EFD0450005000000000079EE00004D660000C9
S113EFE02500FFFF0000000084EE00009180000077
S113EFF02500FFFF0000000088EE0000EDAE0000D9
S113F0002500FFFF000000008FEE0000ADAF000000
S113F01000000000000001000000000000000000EB
S10BF0200000000000000000E4
S113F028FF0000000100000001000000FF040101CE
S113F038B20701008021017001780906FCD57047E8
S90360900C
